:020000040800F2
:10800000384500200181000881DB00086DBE0008B2
:10801000C9DA0008678F00083B0301080000000070
:1080200000000000000000000000000069ED0008F2
:10803000C9A4000800000000F9E0000871FE000873
:1080400017810008178100081781000817810008B0
:1080500017810008178100081781000817810008A0
:108060001781000817810008178100081781000890
:108070001781000817810008178100081781000880
:108080001781000817810008178100081781000870
:10809000AD0201081781000817810008F5AD00083E
:1080A0001781000817810008178100081781000850
:1080B000178100081781000875FE00081781000865
:1080C0001781000817810008178100081781000830
:1080D0001781000817810008178100081781000820
:1080E000178100081781000817810008DFF80CD0FD
:1080F00000F0FEFC00480047251A01083845002022
:1081000005480047FEE7FEE7FEE7FEE7FEE7FEE77D
:10811000FEE7FEE7FEE7FEE7ED80000840EA010328
:108120009B0703D009E008C9121F08C0042AFAD22D
:1081300003E011F8013B00F8013B521EF9D27047F1
:10814000D2B201E000F8012B491EFBD27047002299
:10815000F6E710B513460A4604461946FFF7F0FF46
:10816000204610BD421E12F8013F002BFBD111F832
:10817000013B02F8013B002BF9D17047CAB2401E07
:1081800010F8011F8A4202D00029F9D1002070475F
:10819000421C10F8011B0029FBD1801A704730B532
:1081A00004460020034600E05B1C934203D2E05CDF
:1081B000CD5C401BF8D030BD034611F8012B00F810
:1081C000012B002AF9D118467047F0B480EA010269
:1081D000D40F4200B2EB410F02D2024608461146CC
:1081E0004A0042D0C30DDDB2C1F3C752AD1A202DF3
:1081F00035DAC1F3160141F4000204B15242C5F16F
:10820000200602FA06F12A411044B3EBD05F23D0D6
:10821000C4B1012DA0EBC35009DCF0BC4FF000420B
:1082200002EAC352DBB200F5000000F03FBA4000A2
:1082300000F1807000EBC350A0F1807040EAD17073
:10824000490009E0490841EAC071A0EBC35000F5BC
:108250000000400800EBC350F0BC00F01EBA6142C1
:10826000012202EB4101001BF6E7F0BC704781F0F0
:108270000041AAE780F00040A7E780EA010210B5BC
:1082800002F00043400022D04A001FD0010E01EB53
:108290001261C0F35600C2F3560240F4000042F4EB
:1082A0000002A0FB022000047F39140400D0401C0F
:1082B00050EA124001D44000491EC2B20C0604EB41
:1082C000D010401C4008802A02D003E0002010BDDE
:1082D00020F00100002900DA0020184310BD30B45E
:1082E00080EA010202F0004530F0004221F0004037
:1082F00013D090B1C30DD40DC2F31601C0F3160014
:10830000E41A41F4000140F400027D34914201D3AB
:10831000641C00E04900002C02DA30BC00207047E9
:108320004FF400000023914201D3891A034340080F
:108330004FEA4101F7D151B1914202D14FF00041D2
:1083400005E002D24FF0010101E06FF0010103EB03
:10835000C450284430BC00F0A0B9420005D0C0F39E
:10836000C7525242914201DC0020704700EBC150DD
:1083700070472DE9FE4F81EA030404F0004421F028
:10838000004100944FF0000B23F0004350EA010439
:108390005ED052EA03045BD0C3F30A54C1F30A551A
:1083A0002C44A4F2F3340194A0FB0254C1F3130152
:1083B00041F48011C3F3130343F4801301FB02441F
:1083C00000FB034E840A970A44EA815447EA835724
:1083D000A4FB076802958D0A05FB07854FEA932CDD
:1083E00004FB0C542705029D4FEA065847EA16374E
:1083F000B5EB08056EEB070C870E920E47EA811766
:1084000042EA8312A7FB0201B6EB0B0164EB000406
:108410002B0D43EA0C335E1844EB1C50DA465146F0
:10842000E7FB0201C5F313044FEA0B3343EA14538D
:108430004FEA0432019C43EA0603A4F10C040294BF
:10844000009CCDE900B400F06EF903B0BDE8F08FF8
:1084500000200146F9E7C10F80EAE0700844CA072E
:108460009623002100F022B996230022114600F045
:108470001DB90EB5C10F80EAE0700844CA0700219B
:1084800040F233438DE80E000A460B4600F04BF9EC
:1084900003B000BD0EB540F2334102910021CDE999
:1084A00000110A460B4600F03EF903B000BD00F093
:1084B000004220F00040C10DC0F3160040F400005F
:1084C0007F2901DA00207047962903DCC1F196016B
:1084D000C84001E096398840002AF4D040427047F5
:1084E00020F00040C10DC0F3160040F400007F29C9
:1084F00001DA00207047962903DCC1F19601C840DB
:10850000704796398840704770B5C1F30A5201F040
:1085100000450024C1F3130140F2FF3341F4801100
:108520009A4201DA002070BD40F233439A42A2F22F
:10853000334203DC524200F0A0F800E090402C43AC
:10854000F1D0404270BDC1F30A5210B5C1F313011E
:1085500040F2FF3341F480119A4201DA002010BD4D
:1085600040F233439A42A2F2334203DC524200F01B
:1085700084F810BD904010BD00F0004230F0004083
:108580000AD0C10D01F56071C0F3160042EA015135
:10859000C20840071143704700200146704701F0B0
:1085A000004330B421F0004150EA010206D00A0D28
:1085B000A2F56072C1F31301002A02DC30BC002076
:1085C0007047440F44EAC104C100E01830BC00EB1E
:1085D000C25000F062B80000002801DBC0F100408A
:1085E000002901DBC1F100418142704730B50B46E3
:1085F000014600202022012409E021FA02F59D42D3
:1086000005D303FA02F5491B04FA02F52844151EA6
:10861000A2F10102F1DC30BD2DE9F05F054600203A
:1086200092469B4688460646814640241BE02846E3
:1086300041464746224600F020F853465A46C01AA3
:10864000914110D311461846224600F063FA2D1AC4
:1086500067EB01084F4622460120002100F05AFA3C
:1086600017EB00094E41201EA4F10104DFDC48464F
:1086700031462A464346BDE8F09F202A04DB203AD3
:1086800021FA02F00021704721FA02F3D040C2F132
:10869000200291400843194670470029A8BF70473F
:1086A000401C490008BF20F00100704710B4B0FA28
:1086B00080FC00FA0CF050EA010404BF10BC7047C3
:1086C00049B1CCF1200421FA04F411FA0CF118BFDD
:1086D000012121430843A3EB0C01CB1D4FEA0061AC
:1086E0004FEA102042BF002010BC704700EBC3507F
:1086F00010440029A4BF10BC7047401C490008BFAB
:1087000020F0010010BC704710B5141E73F1000476
:1087100008DA401C41F1000192185B411A4301D173
:1087200020F0010010BD2DE9F04D92469B4611B19D
:10873000B1FA81F202E0B0FA80F22032904600F005
:10874000E9F904460F4640EA0A0041EA0B015346A4
:108750005A46084313D0114653EA010019D0C8F114
:1087600040025046FFF789FF05460E4650465946DF
:10877000424600F0CFF9084305D0012004E020462E
:108780003946BDE8F08D0020054346EAE0762C43EB
:1087900037430A986305E40AA0EB08000022FD0AAB
:1087A00044EA47540A3002D500200146E9E70105B2
:1087B00010196941DDE9084500196941BDE8F04D2E
:1087C000A2E72DE9FE4F804681EA0300C00F0C4668
:1087D000009021F0004123F00045B8EB0200A941D0
:1087E00005D24046214690461C460B46024623F0E1
:1087F0000040104347D0270DC7F30A00C3F30A51C6
:108800000290401A019040286BDAC3F3130040F441
:10881000801B0098924620B10023D2EB030A63EB41
:108820000B0B01985946C0F14002504600F072F916
:1088300006460D4650465946019A00F07AF910EB6B
:1088400008006141002487EA115284EAE7731A4361
:1088500040D0009A62B3019A012A4FEA075215DC10
:10886000001B61EB02014FF0004202EA0752CDE922
:108870000042001C41F5801132462B46FFF753FFA2
:1088800003B0BDE8F08F40462146F9E7001B61EBDD
:108890000201001C41F5801300185B412018A2F56D
:1088A000001747EB030140EAD570B6196D4111E09E
:1088B0006D084FEA360645EAC0754FEA0752001BBD
:1088C00061EB0201001C41F5801149084FEA3000BC
:1088D0000019514132462B4603B0BDE8F04FFFF777
:1088E00013BF0098012240000023D0EB020263EB8B
:1088F000E073009821464FEAE074B8EB000061EBAA
:108900000401E9E783F000435BE781F0004158E7A9
:108910002DE9F04D81EA030404F0004B21F00045FD
:1089200014464FF0000A23F0004150EA050220D01F
:1089300054EA01021DD0C5F30A570246C5F31303DA
:10894000C1F31300C1F30A5640F4801543F48013B9
:10895000A7EB0608101BD64608F2FD3873EB05009E
:1089600002D308F1010801E092185B41B8F1000F51
:1089700003DA00200146BDE8F08D00204FF480119D
:10898000064684460EE0171B73EB050705D3121B42
:1089900063EB050306434CEA010C49084FEA30003B
:1089A00092185B4150EA0107EDD152EA030012D060
:1089B00082EA040083EA0501084305D0101BAB419D
:1089C00006D20122002306E000224FF0004302E01D
:1089D0006FF0010253101AEB06004CEB085110EB3C
:1089E0000A0041EB0B01BDE8F04DFFF78DBE2DE90C
:1089F000F04D00231A461B1A8A4103DB0020014672
:108A0000BDE8F08DC1F30A52C1F3130141F48015A2
:108A10004FF0000BD10702D100186D41521E002704
:108A2000044640F2FF11384601EB620A3E4680469A
:108A3000024600204FF48011FFF71FFEC21971415A
:108A4000BB1846EB0100B4EB030C75EB000C04D330
:108A5000E41A65EB000517460E46241908F10100DB
:108A60006D4180463428E3DDF91946EB0600091B09
:108A7000A84103D24FF0FF32134601E00022134613
:108A80001BEB070046EB0A51BDE8F04DFFF73CBE7B
:108A9000C1F30A52C1F3130140F2FF3341F48011D4
:108AA0009A4202DA00200146704740F233439A426C
:108AB000A2F2334202DC5242FFF7DFBD00F02AB8D7
:108AC00030B5041E71F1000404DB4FF00044404255
:108AD00064EB0101141E73F1000405DB1C464FF02A
:108AE0000043524263EB0403994208BF904230BDF9
:108AF000064C074D06E0E06840F0010394E80700EB
:108B000098471034AC42F6D3FFF7F4FA7C350108ED
:108B10009C350108202A04DB203A00FA02F10020EB
:108B200070479140C2F1200320FA03F319439040AB
:108B30007047202A06DBCB17203A41FA02F043EABD
:108B4000E07306E041FA02F3D040C2F12002914006
:108B500008431946704770B521F0004303430CD019
:108B6000C1F30A550024D5EB040564EB0403D617C2
:108B7000AD1AB34102DB0020014670BD201841EB65
:108B8000025170BD70B58C1810F8015B15F0070329
:108B900001D110F8013B2A1106D110F8012B03E096
:108BA00010F8016B01F8016B5B1EF9D12B0705D49E
:108BB0000023521E0DD401F8013BFAE710F8013BE7
:108BC000CB1A921C03E013F8015B01F8015B521E03
:108BD000F9D5A142D8D3002070BDC94301607047C8
:108BE0000029816802D041F0010101E021F001017A
:108BF0008160704730B587B0012140F2044005F034
:108C0000BDFD4FF4804005F0A3FD5C20ADF81400DD
:108C100000248DF8174005A9164802F0FBFB164DFD
:108C2000284600F02BF84FF46020CDE90204012023
:108C30008DF804408DF8100000948DF805406946C9
:108C4000284600F055F801212846FFF7C9FF2846BD
:108C500000F0ACF8284600F044F80028FAD1284685
:108C600000F0B3F8284600F02BF80028FAD107B03E
:108C700030BD000000080140002801400D4910B53A
:108C8000884202D1012144150AE00B49884202D1F1
:108C90000121041504E0094988420AD10121CC03CD
:108CA000204605F077FD2046BDE81040002105F084
:108CB00071BD10BD0024014000280140003C01406E
:108CC000014600208968490700D501207047C06C23
:108CD00080B270470246002012680A4200D001208C
:108CE0007047014600208968090700D501207047B8
:108CF00010B542680E4B0C791A400B6842EA042208
:108D00001343436082680B4B1A40D1E9024323436B
:108D10004C7942EA440213438360C26A097C22F41C
:108D20007002491EC9B242EA0151C16210BD000081
:108D3000FFFEF0FFFDF7F1FF70B5072609290AD9FC
:108D4000C568A1F10A0404EB4404A640B543A3405E
:108D50001D43C56007E0056901EB4104A640B5432A
:108D6000A3401D4305611F23072A09D2446B521EED
:108D700002EB820293409C4391400C43446370BDDC
:108D80000D2A09D2046BD21F02EB820293409C434E
:108D900091400C43046370BDC46A0D3A02EB820239
:108DA00093409C4391400C43C46270BD816841F084
:108DB0000801816070470029816802D041F4A00158
:108DC00001E021F4A00181607047816841F0040155
:108DD000816070477CB506461421684602F060FE4B
:108DE0000098152184B2684602F05AFE00998DB2AF
:108DF00054B102F031FE012806D16C43C83CA0B248
:108E0000864201D201207CBD00207CBD2DE9F047C7
:108E100015460A4606886421540813464FF0000C94
:108E2000AE427DD300EB4206DFF8048136F8026CD7
:108E30004FF0FF37AE4278D874E0944275D830F8DE
:108E40001460AE422BD200EB440333F8023CAB4239
:108E50001CD900EB4401B0B231F8021CA1EB0000B8
:108E6000FFF7F9FA81463046FFF7FEFA0646284634
:108E7000FFF7FAFA3146FFF7FAF93946FFF76DFACC
:108E80004946FFF72CFA054620462CE004D1A4F110
:108E90000100FFF7E0FA38E0234664443FE001D1E7
:108EA000204630E000EB44067688AE4228D230F807
:108EB000141000EB44004088A1EB0000FFF7CBFA50
:108EC00081463046FFF7D0FA06462846FFF7CCFA2F
:108ED0003146FFF7CCF93946FFF73FFA4946FFF72D
:108EE000FEF90546601CFFF7BFFA3946FFF735FA71
:108EF0004146FFF76AF92946BDE8F047FFF7B7B9E1
:108F00000BD104F10100FFF7AFFA3946FFF725FA5C
:108F10004146BDE8F047FFF758B9A4461C4400E0BD
:108F200003E06408491E89B287D20020BDE8F087BB
:108F3000000080BF10B578B14FF48054012805D0EF
:108F400002280FD11021012006F09CF82146BDE82F
:108F50001040022006F04EB81021BDE8104001205C
:108F600006F090B810BDFEE7C1B2000A40EA012049
:108F70007047000070B55E4B5E4C00205988A4F12C
:108F8000400202E0155C2554401C8842FAD359483F
:108F9000626820301F294260A268826006D00220E9
:108FA000FFF7C8FF00201A21206020E0E07B28287E
:108FB00001D02A280AD1D4F81110227D09BA21F053
:108FC000FF0111435960E18A49BA99604A4A216810
:108FD000914253D1494A617B1268914203D8A17BE7
:108FE00009B110290CD90220FFF7A4FF2421052084
:108FF00006F02EFABDE870400021012006F004BA08
:10900000282860D01DDC1A2849D00DDC0A286AD037
:1090100005DC70B3032836D008282FD163E012286E
:1090200035D015282AD15EE01E2834D004DC1B2858
:1090300031D01D2822D156E0232838D025281DD133
:1090400039E08A284FD00CDC55284CD004DC2A2883
:109050003FD02F2812D142E05A2824D088280DD1A1
:1090600041E0A8283FD005DC8F283CD09E2805D1C0
:1090700039E024E0AA2836D0AF2834D00220FFF708
:1090800059FF2021B3E7BDE8704005F00DBEBDE8F3
:10909000704005F07FBDBDE8704005F011BEBDE831
:1090A000704005F0A9BDBDE8704005F09FBDBDE86A
:1090B000704005F0E9BDBDE8704005F0D3BDBDE8E6
:1090C000704005F001BED3E90101BDE8704005F034
:1090D00099BDD3E90101BDE8704005F013BEBDE8BC
:1090E000704005F0F5BDBDE8704005F067BD0000BB
:1090F000CC010020A8340020555342433402002004
:10910000FEB500270E4604460097880801901E48C9
:109110004169490603D4416941F0400141611B4D59
:109120000120A86008E054F8040B0090009808F0B3
:1091300073FD0090009828600198411E0191F2D2C1
:10914000286808F069FD009006F0030010490190BE
:1091500013E014F8010B009A504000900297009819
:10916000C007009802D081EA500000E0400800905B
:109170000298401C02900828F1D30198421E0192E7
:10918000E7D20098C043FEBD00100240003002400C
:109190002083B8ED2DE9F84F0020ADF800004BF624
:1091A000BF7648F280084A4D4A4C40F68F7ADFF885
:1091B000289148F60F7B494F2FE0088810F00F00E8
:1091C00089F8000032D007EB8001D1F8002CADF80F
:1091D0000020BDF8002012040BD5D1F8002C02EAC3
:1091E0000A02C1F8002C3E4901EB800050F8040C43
:1091F0008047BDF8000000060FD599F8000007EB86
:109200008001D1F8002C02EA0B02C1F8002C35498C
:1092100001EB800050F8040C80472D484430006872
:10922000314908800004C8D4BDE8F88F2868208040
:10923000208800F030006080208800F440502080BA
:109240002868304080F4005080F0200040EA080098
:1092500028600888C00617D4296801EA0B01296034
:1092600003F064F828E02188890401D580F40050D7
:109270006188C90628D46188890601D580F020005C
:1092800040EA08002860CFE72868ADF80000BDF884
:109290000000000506D5296801EA0A01296006F0E8
:1092A000FFF809E0BDF800000004B6D5286800EA20
:1092B0000A00286004F0A2FD286821883040C90413
:1092C000D1D580F48050CEE780F01000D3E70000C5
:1092D000005C0040220300201003002000500040EA
:1092E00010020020F40100202C0200202DE9F041A2
:1092F0003C4C20793C4F0126C7F88461042007F5D7
:10930000C27701F0F1F8032002F092F900258046BF
:109310003D60042001F0E8F8032002F089F9FFF72E
:10932000A3F807464046FFF79FF83946FEF79FFF30
:109330002E49FEF7A2FF2E49FEF79FFF2D49FEF7AB
:109340009CFF6FF00B01FFF708F82B49FEF7C7FFF2
:109350002A49FEF7C4FFFFF7AAF800B2002801DA95
:10936000002004E0B0F5C87F01DDA67003E0A57021
:10937000E179491CE171A178012902D1A179012982
:1093800001D06571A582A178A1711D4BA18A23F836
:109390001100491C88B2A082052801D3A5826671FC
:1093A00061790020002901460BD033F81120491CB7
:1093B0001044C9B200B20529F7D3052190FBF1F0A2
:1093C0000BE0A28A05E033F81150491C284400B292
:1093D000C9B29142F7D390FBF2F060820120BDE860
:1093E000F08100001C0000200000214200404E459A
:1093F00000007A440000C84200B0314500005041EE
:109400002C03002070B50E4800250078012802D0FA
:10941000022802D002E0022600E006260024F0B274
:1094200002F006F9641CE4B20544032CF7D30320D0
:10943000B5FBF0F048F6CC514843000B70BD00007E
:109440006000002040434FF47A72514390FBF1F0EA
:1094500080B2704770B5040018D00846FFF704F8D2
:1094600005462046FFF700F82946FEF706FF0949A2
:10947000FEF735FFFFF780F808F0DCFB0022064B13
:10948000FEF777FFFFF75FF880B270BD46F66050D9
:1094900070BD00000000C84200408F4002F064BB75
:1094A00010B501280BD0022810D13C21A12002F0D8
:1094B00083FD3C21C020BDE8104002F07DBD3C2171
:1094C000A02002F079FD3C21C820F4E710BD000087
:1094D0000749012806D0022808D10871C870002069
:1094E00002F0D6BC012008710020C870704700004F
:1094F0001C00002003490020086034394870C881EE
:109500007047000050000020810008480844D0F84F
:10951000001C490409D5D0F8001C48F68F72114090
:109520004CF280021143C0F8001C7047005000400C
:10953000810008480844D0F8001C490609D5D0F835
:10954000001C48F68F72114048F2C0021143C0F867
:10955000001C704700500040F0B5A3B020258021CA
:1095600002A8FEF7F4FD0024264602AFE006CDE98E
:109570000076010E08238022002004F007FC641C02
:10958000E4B2B4EBD50FF1D323B0F0BD81000648AF
:109590000844D0F8001C48F68F62114048F280025F
:1095A0001143C0F8001C7047005000400A280BD23D
:1095B000064B00EB400203EB82000021416041704A
:1095C000418003F822108160704700005C03002096
:1095D0003CB50225059C09B200B2CDE9004506F074
:1095E0002BF83CBD02464FF400710148FEF7A8BDC0
:1095F0004C3100200A2806D2034A00EB400002EB5F
:1096000080000021417070475C03002008B10448CD
:10961000704704490820096808820020704700004C
:10962000380200201403002008B1044870470449A0
:1096300008200968088200207047000038020020D6
:10964000140300202DE9F34F4FF00008ADF2D44D84
:1096500004464FF480664546C146314609A8FEF7E8
:1096600076FD32462146B148FEF758FD34210DF50E
:109670008D60FEF76CFDDFF8B8B2B24600244421DD
:109680000DF22440FEF763FDA84A0DF224414AE0A2
:10969000505D6D1C0855ADB20A2807D008194078F6
:1096A0000D2803D0B8F1000F3FD138E00020085555
:1096B000084606F053FB9DF8240418B300240DF26D
:1096C00024475BF824603046FEF762FD82B217F84B
:1096D000011BA1F14100192800D8203116F8010B17
:1096E000A0F14103192B00D82030521E1204120C95
:1096F00001D08142EBD0081A104308D0641CA4B2F8
:10970000102CDCD309F1010000F0FF090DE009A8DD
:1097100000EB84100DF22441FEF74EFDF2E7641CCD
:10972000A4B2402C01D25545B2D3B9F1100F01D2E9
:109730005545A3D3B8F1000F0CD1002009A901EBC6
:10974000801212783AB1401C80B21028F7D3B8F1D9
:10975000000F03D0ABE04FF00108A8E00DF58D61DC
:1097600009A807F0F3FF20B100205FEA000802D04B
:109770009DE00120F9E729220DF58D610DF29C4055
:10978000FEF7CCFC9DF891048DF8C504DDF8940437
:10979000CDF8C804DDF89804CDF8CC0424220DF2ED
:1097A000AC416846FEF7BAFC0DF29C4494E80F0009
:1097B00000F052FBBDF86C040A25B0FBF5F35C46E3
:1097C0005CA109A8DBF8002008F092F9BDF86E044E
:1097D00058A1B0FBF5F319A8626808F089F9BDF843
:1097E000700454A1B0FBF5F329A8A26808F080F931
:1097F000BDF872044FA1B0FBF5F339A8E26808F098
:1098000077F9BDF886044BA1B0FBF5F349A82269AE
:1098100008F06EF9BDF87A3446A159A8626908F0DB
:1098200067F9BDF87C3443A169A8A26908F060F922
:10983000BDF878343FA179A8E26908F059F9BDF87C
:1098400080343CA189A8226A08F052F9BDF87E3420
:1098500038A199A8626A08F04BF9BDF8883435A19F
:10986000A9A8A26A08F044F9BDF8823431A1B9A8C8
:10987000E26A08F03DF9BDF884342EA1C9A8226B34
:1098800008F036F9BDF88A342AA1D9A8626B08F02D
:109890002FF9BDF88C3427A1E9A8A26B08F028F9AC
:1098A000BDF88E3423A1F9A8E26B08F021F95146E6
:1098B000DDF8D804FEF74BFC1D4D4FF00004803559
:1098C000B8F1000F12D0A5F14006DDF8D80456F823
:1098D0002410FEF747FC55F82410DDF8D804FEF7F5
:1098E00041FC641CA4B2102CEFD310E009AE06EBCF
:1098F0008411DDF8D804FEF735FC55F82410DDF8A6
:10990000D804FEF72FFC641CA4B2102CEFD3DDF8B2
:10991000D804FEF73DFC094981F81C04000A81F8CF
:109920001D040DF2DC4D4046BDE8F08F802A00207A
:109930008800002025733D2564000000800400207D
:1099400070B5ADF5816D0024ADF8004405F086FDDD
:109950000DF58062111D1AA005F0BCFA1B4E050022
:1099600002D01B48854202D901F0D2FC1BE03470C2
:1099700069462846FFF766FEA8B116480121281A55
:10998000A0F50070C21700EB9250134A02EBA02022
:1099900001706846FEF7FCFB024669462846FEF762
:1099A000BDFB04F0DBFFB068C471047244717068E1
:1099B000C4604461C46184610DF5816D002070BD97
:1099C000434F4E464947202054585400640000201D
:1099D000802A002080040020802E00202DE9F04104
:1099E000ADF58A6D0026ADF840644FF4806168469D
:1099F000FEF7ADFB02210DF5896002F051F8DDF8AC
:109A000048040A2780B2B0FBF7F3FE4CFEA10DF527
:109A10008060226808F06CF80DF580616846FEF7FA
:109A2000A1FB04F1800568462968FEF79BFB032132
:109A30000DF5896002F034F8DDF84804F2A180B237
:109A4000B0FBF7F30DF58060626808F051F80DF592
:109A500080616846FEF786FB68466968FEF782FB10
:109A600004210DF5896002F01BF8DDF84804E6A139
:109A700080B2B0FBF7F30DF58060A26808F038F80B
:109A80000DF580616846FEF76DFB6846A968FEF734
:109A900069FB05210DF5896002F002F8DDF8480444
:109AA000D9A180B2B0FBF7F30DF58060E26808F051
:109AB0001FF80DF580616846FEF754FB6846E968BB
:109AC000FEF750FB16210DF5896001F0E9FFDDF886
:109AD0004804CDA180B2B0FBF7F30DF58060226998
:109AE00008F006F80DF580616846FEF73BFB684616
:109AF0002969FEF737FB07210DF5896001F0D0FFDA
:109B0000DDF84804C0A183B20DF58060626907F0FA
:109B1000EFFF0DF580616846FEF724FB6846696932
:109B2000FEF720FB08210DF5896001F0B9FFDDF893
:109B30004804B5A183B20DF58060A26907F0D8FF93
:109B40000DF580616846FEF70DFB6846A969FEF7D2
:109B500009FB09210DF5896001F0A2FFDDF8480439
:109B6000A9A183B20DF58060E26907F0C1FF0DF590
:109B700080616846FEF7F6FA6846E969FEF7F2FA90
:109B800010210DF5896001F08BFFDDF848049EA1DE
:109B900083B20DF58060226A07F0AAFF0DF580619F
:109BA0006846FEF7DFFA6846296AFEF7DBFA0A2103
:109BB0000DF5896001F074FFDDF8480492A183B2CD
:109BC0000DF58060626A07F093FF0DF580616846CD
:109BD000FEF7C8FA6846696AFEF7C4FA13210DF564
:109BE000896001F05DFFDDF8480487A183B20DF5BF
:109BF0008060A26A07F07CFF0DF580616846FEF781
:109C0000B1FA6846A96AFEF7ADFA14210DF589602C
:109C100001F046FFDDF848047BA183B20DF58060BA
:109C2000E26A07F065FF0DF580616846FEF79AFA73
:109C30006846E96AFEF796FA15210DF5896001F08C
:109C40002FFFDDF8480470A183B20DF58060226B10
:109C500007F04EFF0DF580616846FEF783FA68460F
:109C6000296BFEF77FFA12210DF5896001F018FFCC
:109C7000DDF8480464A183B20DF58060626B07F0E3
:109C800037FF0DF580616846FEF76CFA6846696B30
:109C9000FEF768FA11210DF5896001F001FFDDF88A
:109CA000480459A183B20DF58060A26B07F020FF34
:109CB0000DF580616846FEF755FA6846A96BFEF718
:109CC00051FA17210DF5896001F0EAFEDDF848042C
:109CD0004DA183B20DF58060E26B07F009FF0DF531
:109CE00080616846FEF73EFA6846E96BFEF73AFA8D
:109CF0000DF58862111D46A005F0ECF8474D0400F3
:109D000022D06846FEF744FABDF8401405EB411135
:109D100081F81C04000A81F81D04601BA0F5007086
:109D2000C21700EB925005F5285202EBA02001214A
:109D300001706846FEF72CFA024669462046FEF797
:109D4000EDF904F00BFE57E00DF58862111D34A00B
:109D500005F0C0F8354C364F4FF4185800B30146A3
:109D6000FE226846FEF7DAF941462C48FEF7EFF985
:109D70002BA0FE2201682162416861628068A062B6
:109D8000694604F58060FEF7C9F985F82B64C5F8CB
:109D90003674032085F83A04FE2085F83C0403E07D
:109DA00041461E48FEF7D3F919A0016821604168B9
:109DB00061608068A0601F4801682960416869602F
:109DC0001D4902680A60406848606846FEF7E0F98D
:109DD0000446024669461948FEF7A0F985F80B6467
:109DE000C5F81674022085F81A0485F81C44200A68
:109DF00085F81D0404F0E6FD024924398868C6711F
:109E000006721DE08800002025733D2564000000D7
:109E1000434F4E46494720205458540080040020A8
:109E20004C4F474F494E2020424D500080080020A3
:109E3000188DDD404420010880060020800A0020A3
:109E400046714868C6604661C66186610DF58A6DD7
:109E50000020BDE8F08100000FB4292210B502A94E
:109E60000748FEF75BF99DF83110054880F8291086
:109E70000D99C1620E991838816410BC5DF814FB0D
:109E8000E430002010B5044629220749FEF746F9C0
:109E9000054890F8291084F82910C06AE062024849
:109EA0001838806C206310BDE430002010B586B0F7
:109EB000044614216846FEF74AF9C5F30E0164F31F
:109EC00004011A4B21F49070122219788DF80020A9
:109ED0008DF8012020F4E0408DF8022061F34B2042
:109EE00013228DF80320020B022404EB820444F0B9
:109EF00080048DF804408DF80500000A8DF80600F6
:109F0000FF208DF8070014208DF80800FE208DF842
:109F10000900491C01F0070018700A2000EB8201BB
:109F2000684601F087FF06B0002010BDC001002088
:109F30002DE9F0475DA088B0D0E90010CDE906100A
:109F40000C21684601F0ACFD00980024DFF8648124
:109F5000C5B24FF00509A24606AF6846395D01F06B
:109F600061FE9DF800008DF80C009DF801008DF851
:109F70000D00DDF80200CDF80E00DDF80600CDF88A
:109F80001200BDF80A00ADF816009DF80D0000287B
:109F900078D0385D062872D2DFE800F059655C7130
:109FA00003440DB1022D2CD198F80B00401CC0B217
:109FB00088F80B0002280BD988F80BA0FFF722FACB
:109FC00080B2FEF767FA02460B46002005F0BAF8A9
:109FD00001F042FD022812D11221684601F060FD15
:109FE0000098002186B2684601F05AFD009880B2C0
:109FF0002EB141F66411884201D806F01DFA022DF7
:10A000003DD098F80A00464610B12B4946220A7006
:10A0100005F048FC86F80AA0012D30D1012005F09A
:10A0200085F82CE098F80A00464618B9002001F09F
:10A0300077FAB072B07810BB012001F071FAF0B17C
:10A04000317888421BD03070FFF72AFA17E003F00E
:10A0500055FE14E0012D12D001F092FC02280ED121
:10A06000FFF744F90BE0012D09D001F089FC02282B
:10A0700005D101F073FD01280CD0FFF73BFA385DE4
:10A08000FFF7B8FA641CE4B24C45FFF466AF08B0C1
:10A09000BDE8F087FFF702FA05F066FFFEF7E9F981
:10A0A00002460B46012005F04DF8E8E700040502E2
:10A0B00001000000480100209E0100207CB5FFF750
:10A0C000A1F986B21121684601F0EAFC009800244B
:10A0D00085B201F0C7FC002813DD642190FBF1F08C
:10A0E00081B23046FFF7AEF9084941F288324D435C
:10A0F00095FBF0F0064980B29042488000D94A8032
:10A100007CBD641CE4B2032CE3D37CBD404B4C000B
:10A110006000002018B50023009308E003780C7855
:10A12000A34208D1009B401C5B1C491C0093934236
:10A13000F4D3012018BD002018BD70B586B00546C7
:10A14000072414216846FEF702F812208DF800005B
:10A150008DF801008DF8020013208DF80300288887
:10A160000221C0F3023001EB800040F080008DF846
:10A17000040028788DF8050028886B46000A8DF8C1
:10A18000060000210EE005EB810002791A551A192C
:10A19000467956708679241D9670C079491CD07016
:10A1A000E4B2C9B22888C0F302308842EBD8FF205D
:10A1B0001855181914214170FE21817028880A2130
:10A1C000C0F3023001EB8001184601F033FE06B007
:10A1D000002070BD2DE9F047DFF89490254F4FF037
:10A1E0003008D9F8001001F11005088A0E7A08B974
:10A1F000042E04D0AC88A04215D8042614E01E48D2
:10A200000178012903D00726102038802BE01B4A53
:10A21000002112681A4B120403EBD2325160A7F8E6
:10A22000008001701FE00226844200D90446A9681C
:10A23000204688478246002001F0FAFA014622466D
:10A24000504606F0B5F82146002004F00DFF28889E
:10A25000001B2880688820446880A7F8008009498E
:10A260004FF440500880D9F800000672BDE8F0872E
:10A2700014030020240300200C030020505C004045
:10A2800000600040220300202DE9F047224EDFF855
:10A290008C803027346834F8100FA168A9B100B35E
:10A2A000A588854200D905462846884781462088EA
:10A2B000401B2080608828446080002001F098FACC
:10A2C00001462A46484603F007FF208848B1144952
:10A2D0004FF4405008800021084604F0C5FEA8F85D
:10A2E00000702088A188884201D3032001E020B1BA
:10A2F000052031680872BDE8F087316806200872D1
:10A30000084900200968084A090402EBD131486075
:10A31000A8F80070EFE700001403002024030020D9
:10A3200022030020505C004000600040F8B55D4C06
:10A330005D4D09262068002729684278062A05D045
:10A34000AAB1082A4DD00A2A50D06BE002785206F2
:10A3500068D18078012804D0022804D0032804D0D2
:10A3600060E0C96956E0096A54E0496A52E04288EF
:10A37000B2BBC288022A55D102798ABB0278530641
:10A3800001D1838833B102F07F02012A04D0022A6E
:10A390000CD047E045493DE08A694079002190476B
:10A3A000F0B92068807A0028F4D13BE0417901F0CF
:10A3B0000F0001F070020B063D4901EB8001D1F85E
:10A3C000001C03D5C1F30111090102E0C1F3013101
:10A3D0000903384B1B78834224D90AB90029D9D103
:10A3E00020E0007840061DD1334913E0027802F0E6
:10A3F0007F02012A16D1827AA2B1428892B90279EB
:10A4000082B9C288012A0DD18A694079002190471A
:10A4100040B92A4931B120684782816100208847CC
:10A42000002006E0296820680969407888470328E9
:10A4300013D021680A8AA2F57F43FF3B0BD0022884
:10A440000ED06AB10878000626D5C88800908242EE
:10A450000AD9088218E00E72F8BD20680672F8BDAD
:10A460004FF008000872F8BD0ED22868144B90F81F
:10A470002C00824201D21F7006E0B2FBF0F400FB18
:10A48000142008B901201870286890F82C008882E0
:10A49000BDE8F840FFF79EBE03200872094900039B
:10A4A0000880F8BD14030020180300209DFB00085D
:10A4B00000500040A802002031FB000875FB000896
:10A4C0000C030020220300207047000010B501217A
:10A4D000084604F053F9BDE810400121014800F09E
:10A4E000E7BF00000002300008494A6810444A688B
:10A4F000824203D84A688242FCD370474A680A2ADB
:10A50000FCD84A688242FCD370470000000000205B
:10A5100008B5ADF80000BDF80000411EADF8001010
:10A52000F9D208BD08B50090411E009101D308463C
:10A53000FAE708BD10B54FF4185205490548FDF774
:10A54000EDFDBDE8104010210348FDF700BE0000FE
:10A550000090010880040020802E002010B50B46DA
:10A56000044605F05BFA4FF400718BB1B3F5805FE0
:10A5700011D0B3F5205F12D0B3F5804F13D0A3F5FF
:10A580000042B2F5005F15D80D480A46191804E0DC
:10A590000A460C4901E00A460B49204606E00A46F5
:10A5A0000A49204602E00A4609492046BDE8104013
:10A5B000FDF7B4BD2046BDE81040FDF7C8BD000062
:10A5C000001601084C2001088004002080060020AD
:10A5D000800800202DE9F04F0026ADF2144D0D4605
:10A5E00004466FF007074FF6FF794FF40078B1F596
:10A5F000805F4AD0B5F5205F52D0DFF858A1564FA2
:10A600004FF00109B5F5804F5BD0A5F5004BBBF5C8
:10A61000005F39D8AAF528504619A6F5F4464246F7
:10A6200031462046FDF7BBFD20B13046424621466B
:10A63000FDF774FD022101EB5B20798888427CD113
:10A64000464C69463046FEF7FDFF00287DD168463E
:10A65000FDF79EFD798804EB411181F8DC03000AC7
:10A6600081F8DD03301BA0F50070C21700EB925299
:10A670000AEBA22080F800906846FDF789FD0246AB
:10A6800069463046FDF74AFD5DE042463349FDF735
:10A6900086FD002857D0314D42462146284608E025
:10A6A0002F4942460D46FDF77AFD80B342462146CA
:10A6B0002846FDF733FD2F60686840EA09006860AE
:10A6C00041E0284942460D46FDF769FDF8B1424692
:10A6D00021462846FDF722FDD0468AF80190002544
:10A6E0002068CDF800046068CDF80404A068CDF8B7
:10A6F00008040B221CA10DF58060FDF750FD40B150
:10A700006D1CEDB22034102DEAD346B10AE01AE0F8
:10A7100013E0A07E7880267F87F80190F5E77878AF
:10A72000012802D088F800900DE00020787088F8A9
:10A73000010088F8000006E007E0A5F5FC450AEBFB
:10A74000952181F8019004F009F90DF2144DBDE84E
:10A75000F08F0000802E0020640000208004002084
:10A760008006002080080020434F4E4649472020A5
:10A77000545854007CB5102A069C0DD1102B0BD1D7
:10A780002402E51704EB5574044D05EBE4040025A1
:10A79000CDE9004504F050FF7CBD00006C220108AB
:10A7A0002DE9FC4114460F460546002615E02028F9
:10A7B00018D02D2818D03038C0B20C49C0EB00108A
:10A7C00001EB8000CDE90006182314223946284603
:10A7D00004F032FF14352DB2641C20780028E6D135
:10A7E000BDE8FC810A20E8E70D20E6E7242B0108FC
:10A7F0002DE9FC4114460F460546002611E020389D
:10A80000C0B20A4900EB400001EB4000CDE9000670
:10A810000823062239462846641C04F00DFFAD1DAE
:10A820002DB220780028EAD1BDE8FC81EC22010895
:10A830002DE9FC4114460F46054600260FE020385E
:10A840000949C0B201EB0010CDE90006102308222F
:10A8500039462846641C04F0EFFE08352DB22078F6
:10A860000028ECD1BDE8FC81342501082DE9F04F2A
:10A87000B7B08020349000200246339004203290FC
:10A880004FF0100A002435A93EA004F023FB5FEA34
:10A89000000974D099F8000042286CD199F80100A1
:10A8A0004D2868D199F83600FF2809D199F837006A
:10A8B000FF2805D199F83800FF2801D101203390F5
:10A8C000FEF74AFE3220FFF70FFE0DF1080B02A83B
:10A8D0003499FDF73CFC01250026002002462CE0BF
:10A8E000C6EBC401C91D01FB0A9302F13E015F5C86
:10A8F00080210023DDF8CCC0BCF1000F07EA010C79
:10A9000009D0BCF1000F0FD11BF800C04CEA050CB8
:10A910000BF800C008E0BCF1000F05D01BF8008068
:10A9200048EA05080BF80080401C5B1C4908DBB2B4
:10A93000C0B2082BDED3521CD2B25245D0D3680627
:10A94000761C050EF6B2082EC7D30021CDE900B162
:10A9500032980823001BC0000838C1B20020349A86
:10A9600003F014FA641C3298E4B28442AFD34FF47B
:10A970009670FFF7B9FD37B0BDE8F08FFFE700F044
:10A9800007F8F8E74C4F474F494E2020424D500002
:10A99000F0B5124DADF5037D002001242E2102AB50
:10A9A000A5F50076670204EB4002B2FBF1FC01FB67
:10A9B0001C2216F800C0AA5C82EA0C021A54401C41
:10A9C00080B2B842EFD30020CDE9003020238022AE
:10A9D000014603F0DBF90DF5037DF0BDA41E01086F
:10A9E00002F0F6BF03F01EB87047000010B504492E
:10A9F000052005F081FCBDE81040052004F012BBE5
:10AA0000D83400200EB51A49487801282ED00020ED
:10AA1000009001900290BDF8000020F4E04040F466
:10AA20000042087802F5805260F34B2222F4F07263
:10AA3000803222F01F021032ADF80020BDF8042051
:10AA400022F4F8426FF3080242F40042921CADF87F
:10AA500004200322401CADF8062000F00700087017
:10AA6000012048706846FFF768FB0EBD04200EBD4C
:10AA7000C00100200EB515494878012823D00020D8
:10AA8000009001900290BDF80000142320F4704261
:10AA9000087802F5805260F34B2222F4F072803283
:10AAA00022F01F020A32ADF8002001228DF80720A3
:10AAB000401C8DF8063000F0070008704A706846A8
:10AAC000FFF73BFB0EBD04200EBD0000C0010020BF
:10AAD0000EB50021009101910291BDF8001041F4E2
:10AAE0000042134960F30E32087860F34B2222F4DF
:10AAF000E072803222F03F021132ADF80020BDF842
:10AB00000420401C22F4F04242F4004202F50062AC
:10AB10006FF3080242F48062ADF8042000F00700F1
:10AB20000870012048706846FFF707FB0EBD000063
:10AB3000C00100202DE9F04F0746061D00880024C3
:10AB4000C0F302318A0000F01F03C1B0112B7CD189
:10AB500000047AD5A548921E95B2828807F10208B2
:10AB60004FF001094FF0000A52B1A14F9F4B07F17E
:10AB700058004FF0070B914268D3A3F804A0A2E05D
:10AB8000AC216846FDF7E3FA58212BA8FDF7DFFA60
:10AB9000B8F800009549C0F30800401BC01CC0F382
:10ABA0008F00888080463888ADF8B00000206B4662
:10ABB00045E02BA901EBC00156F82020CA600831FE
:10ABC000970F2DD197052BD081F800909DF8AE20DE
:10ABD0004F460AB98DF8AE70BDF808204FF0320C20
:10ABE000521CADF8082003EB001217734968C1F33B
:10ABF000892707FB0CF7C1F3090101EB810C4FEA30
:10AC00004C0CC2E9047C4FF47A72B7FBF2F24A436F
:10AC100002EB82014900A1420FD90C4601910CE0E0
:10AC20000327B7EB927F08D112F0405F26D0C2F322
:10AC30000172012A22D081F800A0401C80B2B0EB42
:10AC4000950FB6D3BDF8080001E0CDE039E0ADF8CE
:10AC5000AC009DF8AE008DF800006548AC221946A6
:10AC60005830FDF75BFA58222BA96148FDF756FAD8
:10AC7000B8F100007ED0FFF72BFF4CE002270F70E9
:10AC80009DF8AE20032A01D08DF8AE70BDF80820E3
:10AC90004FF0640C521CADF8082003EB0012177340
:10ACA0004968C1F3072707FB0CF75761C1F3474712
:10ACB00007FB0CF7176101F07F013227794391619F
:10ACC000BBE7511A9980002220E006EB820102EBDB
:10ACD0000B0C4B88898803EB014307EBCC0141F84F
:10ACE0000C3F51F804395FEA937818D04FF003080D
:10ACF000B8EB937F08D113F0405F45D0C3F30173E5
:10AD0000012B41D081F800A0521C92B2B2EB950FFA
:10AD1000DBD3008938803548808858B360E00389E8
:10AD2000082B01D8082300E05B1C038100EB0C1307
:10AD30004FF0320883F80C90D1F804C0CCF3892C82
:10AD40000CFB08FCC3F810C0B1F804C0CCF3090C2C
:10AD50000CEB8C0C4FEA4C0CC3F814C049684FF450
:10AD60007A7CC1F3892303FB08F3B3FBFCF3C1F343
:10AD7000090100E02EE04B4303EB83014900A142AF
:10AD8000C2D90C464160BFE74FF0020881F800804D
:10AD900003895B1C038100EB0C1383F80C80B1F872
:10ADA00004C04FF06408CCF3072C0CFB08FCC3F87C
:10ADB00014C0D1F804C0CCF3474C0CFB08FCC3F81A
:10ADC00010C009794FF0320C01F07F0101FB0CF14A
:10ADD000996199E70548042108300170A0F80290B4
:10ADE000002041B0BDE8F08F0120FAE7C00100204B
:10ADF0004C33002010B500F001FA002805D000F017
:10AE0000C1F9BDE8104000F0BFB910BD01490860AC
:10AE10007047000014040140064A014600201268F1
:10AE2000044B0A4014331B680B4202D0002A00D0A6
:10AE3000012070470004014030B51A4A8379016847
:10AE400053B313688B431360111D0B680468A3434D
:10AE50000B60017911440B68046823430B60114BAC
:10AE6000083319680468A14319601C1D216805682E
:10AE7000A94321604179102905D011440A6800686E
:10AE800002430A6030BD19680268114319602168E5
:10AE900000680143216030BD0079104402688A4394
:10AEA000026030BD0004014010B502000C464FF0B6
:10AEB000FF0006D0012A03D100F044FE20600020EC
:10AEC00010BD0020FEF78EFB03A200210C20FFF72F
:10AED000AFFC02F013FFFEE744656D6F204D6F6419
:10AEE000650000000149C860704700000020024072
:10AEF00010B5044680050CD1064800F081F80528FD
:10AF000002D03420FFF7EEFF2046BDE8104000F0ED
:10AF100003B810BDA086010070B505464FF4302679
:10AF2000304600F06DF8042811D1094C206940F03A
:10AF3000020020616561206940F0400020613046D8
:10AF400000F05EF8216941F6FD721140216170BD8B
:10AF50000020024008490420CA68D20701D001201D
:10AF60007047CA68520701D502207047C968C906F0
:10AF7000FBD5032070470000002002400248016911
:10AF800041F08001016170470020024070B5054624
:10AF90000C46074800F034F8052802D03420FFF7AB
:10AFA000A1FF21462846BDE8704000F003B800002C
:10AFB000A0860100F0B506464FF400570D4638460E
:10AFC00000F01EF804280CD1064C206940F0010066
:10AFD00020613580384600F013F82169BA1E11400F
:10AFE0002161F0BD0020024003480249416003494D
:10AFF000416070472301674500200240AB89EFCDD7
:10B0000000B50346FFF7A6FF02E0FFF7A3FF5B1EB4
:10B01000012803D0002B00D1052000BD002BF4D166
:10B02000FAE700000148407870470000C0010020A6
:10B03000AC220149FDF772B8A43300202DE9F84F86
:10B040004D4F4FF0000AA7F10C080646ADF800A0DE
:10B05000B8F8000014460D4610B325B3DFF81C9174
:10B0600099F80100012820D033466A462146284637
:10B0700002F0E8FE002814D107F1F4010A1DC1F81E
:10B0800014A0C1F818A0C1F81CA0C1F820A0167027
:10B09000C2E901545046012E09D0022E17D02CE0EF
:10B0A0000220BDE8F88F0320FBE70420F9E7BDF894
:10B0B000003063F31F700A23B4FBF3F5B4FBF3F322
:10B0C00065F3090063F3932020F070600FE0142310
:10B0D000B5FBF3F363F354203223B4FBF3F363F3D0
:10B0E0000600BDF8003063F31F7020F0F0601061BF
:10B0F0003B68DB0D63F39650106199F8033090893B
:10B100004C46042B20F4E0401ED000F5805020F087
:10B110001F00801C908198F804008109908961F3D8
:10B12000871020F4004020F49071207860F34B21C8
:10B13000401C918100F0070020700320607099F896
:10B14000020001280DD012E000F5005020F01F0091
:10B1500009309081BDF8005008EBC5004068886157
:10B16000D9E7042B03D105490520083108700448AC
:10B17000FEF7E3FF002094E758330020C0010020D1
:10B180005C34002000F097BD10B58EB06A460221F5
:10B19000422000F09EFD9DF8010000F0E0004028F4
:10B1A00002D805200EB010BD6A460221432000F0EF
:10B1B00090FD00980D90BDF834006C4610F4E04FFF
:10B1C00006D0C0F3023081004320A21C00F081FDB4
:10B1D000BDF834000421C0F3023004EB80024320A8
:10B1E000921C00F076FD0421072000F06AFD6846FD
:10B1F00002F06CFC0020D5E700F078BD00F058BDEF
:10B20000054910B54978012903D002F049FE2046CE
:10B2100010BD042010BD0000C0010020FCB428496E
:10B2200000260B460A781D8903F10C01022A07D07B
:10B23000012A24D123486F46D0E9002300202BE0C7
:10B240006A4641F28833344600200EE00F78022F20
:10B2500008D18F689F4205D84F689F4202D31E468F
:10B26000CC6804E0401C80B21031A842EED3C2E9A1
:10B270000064DDE9001209B102201CE00320FCBCDF
:10B2800070470C78012C04D14C68944201D28B6831
:10B290002246401C80B21031A842F2D36FF07040B9
:10B2A000824201D132463346C7E90023DDE900126C
:10B2B0000029E3D0012002B0F0BCFFF7BFBE0000C0
:10B2C000A4330020B43001082DE9F04106461746AA
:10B2D0000D46800502D00120BDE8F081FFF784FE15
:10B2E00000240FE0A00502D13019FFF701FE2988E4
:10B2F0003019FFF74BFE042802D0FFF73FFEEAE7C4
:10B30000A41CAD1CBC42EDD3FFF738FE0020E3E7E0
:10B310002DE9F0474FF418512C48FCF718FF2C4842
:10B320002CA12A4E0A6802604A68426089688160DE
:10B330002B48DFF8B08000250168316041687160FA
:10B3400006F5007102680A60406848602C4608F102
:10B350004009474658F82400FCF71AFF02467019C6
:10B3600057F8241000F5C060FCF7D8FE57F8240009
:10B37000FCF70EFF05444F4659F82400FCF708FF80
:10B380000246701957F8241000F5C060FCF7C6FE9D
:10B3900057F82400FCF7FCFE641C0544102CD8D39D
:10B3A000002086F80B041048C6F81604022086F820
:10B3B0001A0486F81C54280A86F81D0404F04EF876
:10B3C00003F000FB0020BDE8F087000080040020AF
:10B3D00080080020434F4E464947202054585400CF
:10B3E00044200108C8000020188DDD4010B58A07F0
:10B3F00021F003040649120F21440F238C68934067
:10B400009C438C608B68904003438B6010BD0000B0
:10B4100000000140F0B5CC78002204F00F03E406F0
:10B4200001D58C7823430C784FF00F0C14F0FF0FEC
:10B430004FF0010E1BD005680E880EFA02F426406C
:10B44000A64210D196000CFA06F725EA070703FA80
:10B4500006F5CE783D43282E02D0482E02D002E0D9
:10B46000446100E00461521C082AE5D305600A88A3
:10B47000FF2A1CD94468002202F108060EFA06F5DC
:10B480000E882E40AE420ED196000CFA06F7BC4351
:10B4900003FA06F7CE783C43282E00D14561CE78DA
:10B4A000482E00D10561521C082AE5D34460F0BD46
:10B4B000F0B5144C002801DAE36900E06368450D3B
:10B4C0002E0185B2C0F30157B540C0F30342032FEC
:10B4D00005D0C6020AD503269640B34307E023F001
:10B4E0007062636823F07063636002E0AB4343F013
:10B4F000706201B12A43002801DAE261F0BD6260A6
:10B50000F0BD0000000001400246002092680A429F
:10B5100000D0012070474161704701617047000011
:10B52000F0B506463F4889B003AB07C883E807007B
:10B530000024172106A800F0B3FA0698C0B2411EF5
:10B54000042905D803A901EB400010F8020C01E022
:10B55000BDF812000C22C5B26946032000F014F9B0
:10B56000DDE900014042CDE90010024606A8029B39
:10B5700000F09CF99DE80E0006A800F097F92A4F0C
:10B580002A4B97F805C0BCF1000F0DF1180C9CE890
:10B59000070007D04FF0000C87F805C003F10C0C32
:10B5A0008CE8070016B1012E22D035E01F4F0C3772
:10B5B0003E68A6EB050C604503DB06EB050C604519
:10B5C00000DD01247E68A6EB050C614503DB06EB7C
:10B5D000050C614500DD641CBE68771BBA4202DBC6
:10B5E0003544AA4200DD641C022C15D2002413E06D
:10B5F000B7F910506E42B14206DAB7F90E607642E2
:10B60000B04201DA022407E0A94205DDB7F90E5085
:10B610006D42A84200DA01240C3383E8070009B028
:10B620002046F0BD6C2E010848010020CC300020DF
:10B6300070B50D4C0146072301222046FDF77CFB27
:10B6400001212046FDF7B7FB02212046FDF742FB12
:10B650000028F9D02046FDF73AFB05460221204696
:10B66000FDF7BBFA284670BD002801400FB4002149
:10B670002DE9F04F8246BDF830C0DDF8D4B00E465B
:10B680000DA8BCF10A0F02D9CAF800602CE000270F
:10B6900026E00278022A20D1C268642402FB0BF360
:10B6A000B3FBF4F5D0E9014399460B9B4FF47A784C
:10B6B00003FB08F3B3FBF4F3A54205D3A1420CD27C
:10B6C000214606E0164608E04D4506D3A94204D2BD
:10B6D00029469342F6D81A46F4E77F1CBFB21030D1
:10B6E0006745D6D3CAF80010CAF80460BDE8F00F69
:10B6F0005DF814FB014880787047000008000020C6
:10B7000070B500220546104611461346012606FA7A
:10B7100003F42C4204D1012906D0032906D006E007
:10B7200041B1022908D008E0022100E00421521CA6
:10B73000D2B206E0012100E00321824200D9104686
:10B7400000225B1CDBB2202BE1D3E90702D182424D
:10B7500000D9104670BD000070B500252C460420AD
:10B76000FFF766FF641CE4B20544032CF7D3032003
:10B77000B5FBF0F0BDE8704082B2A3210148FDF7AF
:10B7800045BB0000FC1E01082DE9FC4105460020D8
:10B7900016460F460190FF24042201A90120FFF75D
:10B7A00083FBDFF844C035B1012D04D0022D09D050
:10B7B000032D0FD111E0019800900C4B3246394611
:10B7C000012005E001980090084B324639460220DE
:10B7D000E04704462046BDE8FC8101980090034BF9
:10B7E000324639460320F3E701200008BC0100205F
:10B7F0000549096889B201EBC000044901EB40002A
:10B80000008980B270470000505C0040006000403A
:10B810000549096889B201EBC000044901EB400009
:10B820008089C0F309007047505C00400060004010
:10B830000449096889B201EBC000034931F81000DE
:10B8400080B27047505C0040006000400FB400239D
:10B850002DE9F0431E46DDE9338CBDF828700A2F30
:10B8600005D906604660BDE8F0035DF814FB0022D0
:10B870000DF1200914E009EB0215297B01290DD1F6
:10B88000D5E90414884509D364254D43B5FBFCF57F
:10B89000A54203D88B4201D20B462646521C92B2D7
:10B8A000BA42E8D3C0E90036DDE700002DE9FF5FCA
:10B8B000DFF8B4A099460024BAF81400DFF8ACB061
:10B8C00000EB40030F460BEB8301401C9046AAF8A7
:10B8D000140081E8800325469AF804002E4638B308
:10B8E0002348244905F0E4FEFCF759FE0A21FCF741
:10B8F00034FDFCF7DCFDAAF80E001F481F4905F0D7
:10B90000D7FEFCF74CFE0A21FCF727FDFCF7CFFD24
:10B91000AAF8100000205A4600EB400102EB81011A
:10B92000401C81E8800310F0FF00F5D08AF8044045
:10B93000BAF8141009B1AAF8144000205A4600EBD6
:10B940004001401C52F8213002EB81011C444B683D
:10B95000896800041D440E44000CF0D0009880E873
:10B960007000BDE8FF9F000048010020CC3000209F
:10B97000EA9DF7ECA6F1F43F557E2C5752C1F03FFB
:10B9800001480079704700001C0000200148C07881
:10B99000704700001C0000200148B0F910007047FB
:10B9A0001C00002003490878002801D000220A70FA
:10B9B00070470000080000200FB40023F0B53C25BC
:10B9C000129EDDE913100122F61F40F2E734102E1B
:10B9D00034D2DFE806F0080808210818181B1F1DDC
:10B9E0000823251F2B2FBDF82C2022B14FF43C72C9
:10B9F0000A807A2103E04FF4C8720A803221018064
:10BA0000F0BC5DF814FB0C800580F9E70A2312E016
:10BA1000022310E00A800BE019230CE00622F9E76C
:10BA20004FF47A620A8040F6B831E8E72D22F1E758
:10BA30000380E5E705230B800280E1E70B80F7E751
:10BA40000148006870470000380300200148408A20
:10BA5000704700004801002001480078704700004E
:10BA6000600000200148B0F9120070471C0000205F
:10BA70000148C07870470000480100201CB505212E
:10BA8000684600F00DF8009884B20448408A00F03F
:10BA9000EFF8844200D820461CBD00004801002079
:10BAA00010B504460020182936D2254A34D2DFE8E2
:10BAB00001F00C0E121416181A27292B2D1D1F2207
:10BAC000242F363A383C3E404244118800E05188E9
:10BAD00061F30F0020E09188FAE7D188F8E7118937
:10BAE000F6E75189F4E7FFF7ABFF15E0D06813E004
:10BAF00092F829100EE0D06A0EE0114830300BE0C9
:10BB0000518AE5E7918AE3E7118AE1E7D18ADFE725
:10BB100092F8281061F30700C4E9000510BD118BED
:10BB2000D6E7518CD4E7918CD2E7118CD0E7518BBA
:10BB3000CEE7918BCCE7D18BCAE7D18CC8E7000068
:10BB4000E4300020014840687047000000000020F9
:10BB500001480078704700001C00002001488078F0
:10BB6000704700001C0000202DE9F0410025FFF780
:10BB7000F3FD064600240320FFF75AFD641CE4B2DF
:10BB80000544082CF7D31848EC088088201A00B226
:10BB9000FCF761FC05461549FCF76FFB0746284694
:10BBA0001349FCF76AFB2946FCF767FB3946FCF7AB
:10BBB0000CFB1049FCF709FB3146FCF706FB0E4F66
:10BBC0003946FCF75AFBFCF772FC05B239463046A1
:10BBD000FCF753FBFCF76BFC03493839C8820C8334
:10BBE0002846BDE8F081000054000020CDCC0C3E7A
:10BBF000ACC5A7B6AC1CC6C00000204170B500257E
:10BC00002C460320FFF714FD05440A20FEF76CFCC8
:10BC1000641CE4B2052CF4D30520B5FBF0F080B22F
:10BC200070BD00000A290DD300210A7802704978FE
:10BC3000417002210A68C0F802204A68C0F8062054
:10BC4000098911E001EB4102084901EB82010A7800
:10BC500002704A784270D1F80220C0F80220D1F870
:10BC60000620C0F806204989418170475C03002006
:10BC70001CB501000AD001290AD0022805D10421EF
:10BC80006846FFF70DFF009880B21CBD0221F7E760
:10BC90000321F5E708B10448704704490120096809
:10BCA00008820020704700003402002014030020A6
:10BCB0008020FFF7B1B810B58020FFF7A7F800206B
:10BCC00010BD0A4610B50146222000F0D7FA002028
:10BCD00010BD10B5144603462222204600F012FA89
:10BCE000002010BD0146222000F0EAB97FB50024F3
:10BCF00000F0B2F90121092002F040FD48208DF842
:10BD00000F008025ADF80C5003208DF80E0003A91C
:10BD10004748FFF77FFB07210120FFF767FB0095EE
:10BD200001258DF8065000208DF804000C208DF8B8
:10BD300005006846FFF780F817208DF808008DF899
:10BD400009508DF80A508DF80B5002A801F026FF1B
:10BD500003210C20FFF7B5FF3220FEF7C5FB0321BE
:10BD60000C20FFF7AEFF0A20FEF7BEFB0F210B20D1
:10BD7000FFF7A7FF4FF496760AE04DB100254FF08C
:10BD800003014FF002002DB1FFF79BFF072104E0F4
:10BD90000125F4E7FFF795FF0B210220FFF791FF44
:10BDA0000120FEF7A1FB4020FFF79CFF00F00F00F1
:10BDB000012806D8641CA4B2B442DED9012004B024
:10BDC00070BD07210920FFF77CFFEF210A20FFF754
:10BDD00078FFEF210E20FFF774FF01210F20FFF7FE
:10BDE00070FF2DB107210220FFF76BFF252104E032
:10BDF0000B210220FFF765FF26210320FFF761FFDB
:10BE000002210C20FFF75DFF00210620FFF759FFFC
:10BE10000F210B20FFF755FF3E20FFF763FF3F2068
:10BE2000FFF760FF4220FFF75DFF0020C7E700003B
:10BE3000000C014070B50C4605460F210B20FFF7A2
:10BE400040FF40210620FFF73CFFE1B243232222BE
:10BE5000284600F02DFA05210620FFF732FFBDE845
:10BE6000704007210B20FFF72CBF00000020FDF7DA
:10BE7000B9FB04A208211C20FEF7DAFC01F03EFF0A
:10BE8000FEE7000048617264204661756C74000032
:10BE9000024900B10120C1F8800170470000214231
:10BEA00038B50121042002F069FC0120ADF8000042
:10BEB00010208DF803000320054C8DF80200694620
:10BEC0002046FFF7A7FA01212046FFF724FB38BDE3
:10BED000000801400020FFF7DBBF00002DE9FC4116
:10BEE000334CC8B102283AD10F216846FFF7D8FD7C
:10BEF0000C216846FFF7D4FD00980026C5B2207BD0
:10BF0000401CC0B2207303283FD3FDF7EFF9608ACD
:10BF1000012D80B225D037E0FFF726FE054602F05E
:10BF200009F92082284604F01FF8FCF7A2FA02461D
:10BF30000B46012003F006F9208A80B202F032FF9E
:10BF4000FFF700FE216B401A02F024FFFFF7FAFD15
:10BF50002063208A08B1012000E00220E070BDE8E3
:10BF6000FC81B0F5C87F0ED2E07A401CC0B2E0720E
:10BF7000022809D3E67202F0D2FD00220D4B0D20FB
:10BF800003F0E0F800E0E6722673FDF73BFA87B2B3
:10BF90003846FCF77FFA02460B46002003F0D2F841
:10BFA000012D02D1384604F0EBFAE670D7E7000025
:10BFB0001C0000200000104070B50C46054603F040
:10BFC000F3FB6006000E03F025FC002003F022FCCA
:10BFD000284603F01FFCBDE8704003F0FDBB2DE9CF
:10BFE000F0419046069E0D460446002703B14027C7
:10BFF00003F0DAFB4FEA4860000E03F00BFC384612
:10C0000003E0012E0AD014F8010B03F003FC6D1EAF
:10C01000EDB2F6D2BDE8F04103F0DEBB2078C043BC
:10C02000C0B203F0F7FB641CF1E7000010B5094A49
:10C030000024C2F89841C2F89441204602F5CA7221
:10C04000FEF770FA012050600020FEF76BFA546092
:10C0500010BD00000080214208B50121082002F037
:10C060008DFB6020ADF8000014208DF80300032044
:10C070008DF8020069460548FFF7CCF90448012114
:10C08000C0F89811C0F8941108BD0000000C0140E0
:10C090000080214230B5094A0025C2F89851012498
:10C0A000C2F89441284602F5CA72FEF73BFA546082
:10C0B0000020FEF737FA556030BD000000802142B5
:10C0C00030B50D46044600F093F86006000E00F00F
:10C0D00071F800F0B7F8284600F06CF800F0B2F8FC
:10C0E00000F086F8012000EB4400C0B200F062F8D6
:10C0F00000F0A8F8002000F031F8044600F08EF8B7
:10C10000204630BDF0B51F4616460D46044600F0E9
:10C110006FF87006000E00F04DF800F093F8384606
:10C1200000F048F800F08EF800F062F8012000EB13
:10C130004600C0B200F03EF800F084F807E00DB110
:10C14000012000E0002000F009F804F8010B6D1E4A
:10C15000EDB2F4D2BDE8F04000F060B82DE9F04156
:10C16000134D002401268046C5F8946122462746D7
:10C17000C5F898710020FEF7D5F9C5F898616006FA
:10C18000040ED5F8140108B1641CE4B20020FEF7D7
:10C19000C9F9521CD2B2082AEAD3B8F1000F04D070
:10C1A000FFF744FF2046BDE8F081FFF773FFF9E792
:10C1B00000802142F0B50D4D00260446C5F8986177
:10C1C00032460127E009C5F894016006040E0020FC
:10C1D000FEF7A8F9C5F898710020FEF7A3F9C5F895
:10C1E0009861521CD2B2082AECD3F0BD00802142E3
:10C1F000094A10B50120C2F89401C2F89801002044
:10C2000002F5CA72FEF78EF9002414602046FEF78C
:10C2100089F9546010BD000000802142084A10B521
:10C220000020C2F89801C2F8940102F5CA72FEF724
:10C2300079F9012454600020FEF774F9146010BDF0
:10C240000080214230B50C4C01221546C4F89421DF
:10C250000020FEF767F9D4F8140100B90022C4F8F1
:10C2600098510020FEF75EF90020C4F89801FEF70F
:10C2700059F9104630BD00000080214270B51546C6
:10C280000E460446FFF7B4FF6006000EFFF792FF6C
:10C29000FFF7D8FF3046FFF78DFFFFF7D3FF2846A3
:10C2A000FFF788FFFFF7CEFFBDE87040FFF7B6BF8E
:10C2B000F0B51E4617460C460546FFF799FF78066F
:10C2C000000EFFF777FFFFF7BDFF304601E015F8DE
:10C2D000010BFFF76FFFFFF7B5FF641EE4B2F6D264
:10C2E000BDE8F040FFF79ABF02494CF6CC40086029
:10C2F000704700000030004002494AF6AA2008605A
:10C30000704700000030004001494860704700005D
:10C310000030004001498860704700000030004054
:10C3200001490860704700000030004010B5134C10
:10C330002068017A022904D0042902D0062905D0F8
:10C3400015E0FDF747FF2068007A11E041780529E4
:10C3500009D10178490606D1C07802F0F7FD0848F6
:10C360000068006A804707480068806880470820A6
:10C3700021680872BDE8104001F0BABF1403002024
:10C380001C0300201803002070B50024FDF73AF8C4
:10C3900085B22846FCF77EF802460B46002002F0E4
:10C3A000D1FE42F23410114E854205D200223346AE
:10C3B0000D2002F0C7FE012447F61810854207D968
:10C3C00000224FF080430D2002F0BCFE44F0040434
:10C3D0002846FCF7FFFC30B1002233460D2002F066
:10C3E000B1FE44F00804204670BD00000000F03F9C
:10C3F0007FB50C4605460121042002F0B3F9ADF8E3
:10C400000040ADF804500024114DADF80640ADF8E1
:10C4100002406946284603F059FD0121284603F0F1
:10C4200035FD01221146284603F047FD012128462B
:10C4300003F039FD1E208DF80C008DF80D40012011
:10C440008DF80E008DF80F0003A801F0A7FB7FBD4B
:10C45000000800401CB504460C216846FFF720FB8D
:10C46000092C0AD2FFF704FB012801D0034804700D
:10C47000BDE81C40022002F05FBE1CBD0800002089
:10C480002DE9F04FA7B082461220FE4E24900621DF
:10C49000F47B6846FFF7C6FB00982922C0F3072803
:10C4A000F94917A8FBF73AFEF74F97F829008DF8DE
:10C4B0008500F86A2290386B239026A825A9CDE93B
:10C4C0000A10242209941BA96846FBF727FE17AD22
:10C4D00095E80F00FFF770FAF079002518B1F571B3
:10C4E0003846FDF7CFFC4FF00109182C19D0172C56
:10C4F00017D03079022814D00020FDF773F8307976
:10C5000001280ED110231A46194602200095FEF785
:10C5100031F910231A4619467020CDF80090FEF725
:10C5200029F9E01F0146009014204FF00A0B122950
:10C5300074D2DFE801F0091A3445546574829DAC69
:10C54000BBCCDBEFFEECEBEA307830B13570388CE9
:10C55000B082B988B1FBFBF07082CCA2002102202E
:10C56000FEF766F90122249B0FE0307830B1357078
:10C57000388CB082F988B1FBFBF07082C5A2002133
:10C580000220FEF755F9249B0222C4A10CA804F056
:10C590007FF80CAA00215820FEF74AF91FE23078F4
:10C5A00030B13570388CB0823989B1FBFBF07082C4
:10C5B000BCA200210220FEF73BF90322249BE4E702
:10C5C000307820B13570A6F81490388C7082B7A2FC
:10C5D00000210220FEF72CF90422249BD5E73078B5
:10C5E00030B13570388CB0827989B1FBFBF0708244
:10C5F000B1A200210220FEF71BF90522249BC4E70B
:10C60000317819B13570B082788A7082ADA200217C
:10C610000220FEF70DF90622249BB6E7DDE1317812
:10C6200019B13570B082B88A7082A9A200210220A7
:10C63000FEF7FEF80722249BA7E7307820B135707B
:10C64000A6F81490388A70823079012808D1317A9E
:10C65000B6F91200814203D0C0B2307201F05CFB27
:10C660009EA200210220FEF7E3F80822249B8CE71B
:10C67000307820B13570A6F81490388B70829AA269
:10C6800000210220FEF7D4F80922249B7DE73078B0
:10C6900020B13570A6F81490F88A708295A2002116
:10C6A0000220FEF7C5F80A22249B6EE7307830B1ED
:10C6B0003570388CB082F98BB1FBFBF0708290A2A0
:10C6C00000210220FEF7B4F80B22249B5DE73078AE
:10C6D00020B13570A6F81490788B70828BA200215F
:10C6E0000220FEF7A5F80C22249B4EE7307820B1FB
:10C6F00035706420B082B88B708287A2002102203E
:10C70000FEF796F80D22249B3FE7A0E02FE01FE004
:10C710000FE0FFE7307820B13570A6F81490788CE0
:10C7200070827FA200210220FEF782F80E22249B55
:10C730002BE7307820B13570A6F81490B88C708251
:10C740007AA200210220FEF773F80F22249B1CE737
:10C75000307820B13570A6F81490F88C708275A2EC
:10C7600000210220FEF764F81022249B0DE73078A8
:10C7700000B1357072A200210220FEF759F8112293
:10C7800046A10CA8249B03F083FF0CAA002158208B
:10C79000FEF74EF83079012802D0022822D021E19C
:10C7A000B8F1000FFBD0B079401CB071707918B1AE
:10C7B000102166A21C2002E067A210211420FEF7BF
:10C7C00037F8707940B100207071B079062805D231
:10C7D00001234FF4FA722AE00120F5E7B571757173
:10C7E000357121E0B8F1000F4AD0B079401CB0712A
:10C7F000707930B3B07A012802D0022804D00AE060
:10C80000102158A21C2002E059A210212C20FEF772
:10C810000FF87079C8B100207071B0790628D7D3AD
:10C82000B57175713571B572012342F2107206212E
:10C8300001A802F085FD4FF000080620FCF7DAFEA3
:10C84000CDE0102144A21420E1E70120E4E7307894
:10C8500000B1357048A200210220FDF7E9FF122245
:10C860000EA10CA8249B03F013FF0CAA0021582052
:10C87000FDF7DEFF3079012802D1B8F1000F7FE02B
:10C88000AAE000009C0100201831002054312054FF
:10C89000656D700054322054656D70002532642F30
:10C8A0002564000054332054656D700054656D702C
:10C8B0002053746570000000536C656570205465EA
:10C8C0006D700000536C6565702054696D650000E3
:10C8D00049646C652054696D650000004261636BBA
:10C8E0006C6967687400000054656D70556E6974FA
:10C8F00000000000446973706C6179446972000043
:10C90000426F6F737454656D70000000506F7765EF
:10C9100072537263000000004D696E566F6C7400B4
:10C920004C6F7743757272656E7400005044507797
:10C930004D6178004D73656E556E6974000000009E
:10C9400054656D7043616C6962000000436F6D70E7
:10C950006C657465640000002020202020202020C9
:10C96000202020004F7665722074656D70000000F5
:10C970004E6F207469702100526573746F72650088
:10C980002AD0B079401CB071707920B1AFF2440266
:10C9900010211C2002E0FEA210211420FDF748FF08
:10C9A000707940B100207071B079062805D201235A
:10C9B0004FF4FA7207E00120F5E7B5717571357132
:10C9C000012342F210720621684602F0B9FC4FF0D2
:10C9D00000080620FCF70EFE56E0182C54D03079E3
:10C9E000022851D00098ED49009111287CD2DFE84F
:10C9F00000F00909097B0912127B1C2909347B3BD1
:10CA00006F7B4200388BB6F9122088BB53E04E2072
:10CA100002F012FE05E0B6F91220E1A10FA803F022
:10CA200037FE10210FAA362012E0708A40B1032091
:10CA3000102300901A4619463820FDF79BFE23E08C
:10CA40000220F5E7708A012805D0D7A210212C20FA
:10CA5000FDF7EEFE18E0D6A2F8E7B6F912200AB10B
:10CA6000D5A13AE0D5A23CE0708A10B1D4A238E05A
:10CA700016E0D4A235E0012102A8FFF711F80298D0
:10CA800001B27182307910B1B07988B35FE1388B2F
:10CA900078B1012003F0A0FA00B290FBFBF27082A3
:10CAA000C9A10FA803F0F4FD10230822194601952F
:10CAB000ADE791FBFBF2C4A10FA803F0E9FDB74875
:10CAC00010231038CDE90005082219469FE70BE036
:10CAD000B6F91220002ACCD0BCA10FA803F0D8FDD3
:10CAE0000FAA10213820B3E7B6F91220B9A195E7B3
:10CAF000FFE741F28832BAF1010F0DD0BAF1020F0F
:10CB00003AD01221BAF1040F7ED0BAF1050F7CD0D1
:10CB1000BAF1070F7AD014E13079012801D0E8B1D9
:10CB200012E1708AB18A401A01B27182BDF8980090
:10CB3000814200DA7082122C02D0152C07D00BE053
:10CB4000B6F91200012806D0022804D004E0B6F994
:10CB50001200122800DA7582012311E1641EE4B28A
:10CB6000062C00D8182486F800900020FCF73AFD27
:10CB7000204602F0CDFA00E13079012801D018B347
:10CB8000E2E0708AB18A401A01B27182BDF8980061
:10CB9000814200DA7082122C02D0152C07D00BE0F3
:10CBA000B6F91200012806D0022804D004E0B6F934
:10CBB0001200122800DA758201230621684602F06D
:10CBC000BFFB01F09BF8BCE0172C23D086F8049043
:10CBD00001230621684602F0B3FB182C41D186F8E8
:10CBE0000990B57186F80590F98A4846012906D062
:10CBF0007A4908707A4908700120FCF751FC79489D
:10CC000001F06BFF012302E035E056E0A9E04FF4AC
:10CC1000FA72B5E0B6F912A0FEF724FF0390B571E1
:10CC20004FF4FA7B86F8059001235A4606216846A0
:10CC300002F086FB388B012805D15146002003F015
:10CC4000CBF90FFA80FADA450CDA0398B0F5C87F11
:10CC500008DDFEF7D3FF86F8049002F0A9FB02F08E
:10CC60001DF96EE002203071DA4502DB86F80A9089
:10CC70006AE0B07268E03079012821D0B0B163E099
:10CC8000122C0AD0152C7FF45AAFB6F91200401EB0
:10CC90001128BFF454AF71825EE7B6F91200012883
:10CCA00001D00228F8D10320708255E7641CE4B259
:10CCB000192CFFF458AF072455E7307901280AD121
:10CCC000708AB38A184403B27382BDF89400834219
:10CCD000D6DD7082D4E7B8BB86F8079086F800905E
:10CCE0000020FCF77FFC29223E4917A8FBF716FA23
:10CCF00097F829008DF88500F86A2290386B239008
:10CD000024221BA96846FBF709FA0DF15C0A9AE890
:10CD10000F00FDF7A1F8FCF761FE707A012802D13F
:10CD2000757202F023F8002002F0F2F90022134697
:10CD30000C2002F007FA0620FCF75CFC0620FCF74A
:10CD400035FC3079012800D0002002F0DBF9B8F181
:10CD5000000F72D03079C0B101285BD0B079A8B192
:10CD60006BE030790128B6D13571182C05D0708A66
:10CD7000214682B21B4802F01DF8012342F21072D4
:10CD80000621684602F0DCFADBE72DE04DE000000A
:10CD90002020202020202020202000002425010801
:10CDA00025336453200000004C65667420000000A9
:10CDB0005269676874000000256453004443000012
:10CDC0004F4E00004F46460025336400256457202F
:10CDD0000000000025336420000000004A0100200C
:10CDE000480100201831002086F8079086F800904E
:10CDF0000020FCF7F7FB002002F08AF9002213461E
:10CE00000C2002F09FF90620FCF7F4FB0620FCF74B
:10CE1000CDFB12E03571708A214682B2094801F0DB
:10CE2000C9FF0020FCF7DEFB00E03571012342F270
:10CE300010720621684602F083FA00F05FFF27B007
:10CE4000BDE8F08F18310020F0B58F4C97B0054643
:10CE5000E67B062110A8FEF7E5FE072113A8FEF7E2
:10CE6000E1FE0027002E45D0022E7DD0012E7CD180
:10CE7000207800287AD0FEF7F5FDFBF7ECFA06469D
:10CE800001216846FEF70CFE0098277005B2FCF7FA
:10CE9000B9FA07B23846FBF7ECFA02460B46002017
:10CEA00002F050F9FEF75AFE784C002877D0784906
:10CEB0003046FBF714FAFBF75FFB02460B4675A101
:10CEC00002A803F0E5FB02AA00210220FDF7B0FC56
:10CED0003846FBF7C0FA2146FBF701FAFBF74CFB9B
:10CEE0000A2295FBF2F2CDE900016DA102A803F040
:10CEF000CFFBC2E008210AA8FEF794FE9DF84D0082
:10CF000038B1A07B401C00F00300A0730820FCF7A0
:10CF100071FB07210DA8FEF785FE9DF834008DF802
:10CF200028009DF835008DF82900DDF83600CDF891
:10CF30002A00DDF83A00CDF82E00BDF83E00ADF82D
:10CF400032009DF8290010B9E078012809D1E77076
:10CF50000020FCF747FBA07B02F0D6FA0720FCF785
:10CF600049FB0126012D02E057E016E064E017D0EE
:10CF700040F6B837022D4AD0042D37D0052D0CD1FC
:10CF800026700020FCF72EFB022002F0C1F80123DE
:10CF90003A4606210DA802F0D3F917B0F0BD59E0CA
:10CFA0000220FCF795FAFCF7A1F9FEF75BFDB0F55E
:10CFB000C87F05DA00223E4B0D2002F0C3F8ECE7F3
:10CFC000022001F07BFDFFF7DFF90028E5D1267094
:10CFD000FCF708FB032002F09BF80022354B0C20E5
:10CFE00002F0B0F8012002F08DF8D6E7267000209C
:10CFF000FCF7F8FA072002F08BF800224FF080438C
:10D000000C2002F09FF8012341F28832C1E726701C
:10D010000020FCF7E7FA0120B7E7207860B127701D
:10D020000020FCF7DFFA24A225A102A803F030FBC0
:10D03000102102AA0F2023E09DF841000028ACD067
:10D040000020FCF7CFFA002002F062F80620FCF77F
:10D05000D1FAA2E71CA200210220FDF7E9FB384625
:10D06000FBF7F9F92146FBF73AF9FBF785FA024697
:10D070000B4617A102A803F00BFB02AA1021022005
:10D08000FDF7D6FBD8E700009C01002000007A44A1
:10D090000000C842546970523A252E3166000000E3
:10D0A00054656D703A256420563A252E3166560037
:10D0B000000010400000F03F56322E3031000000DA
:10D0C0005665723A25730000546970523A2D2D004E
:10D0D00054656D703A2D2D20563A252E3166560036
:10D0E0002DE9F04FDFF870A491B004469AF80F6074
:10D0F00006210AA8FEF796FD10216846FEF7D0FC2F
:10D1000000980B2105B26846FEF7CAFC4FF00A08EA
:10D110004FF0010B4FF00009032E20D0042E7CD1DC
:10D1200013216846FEF7BCFC0098002D86B275D02E
:10D130004FF47A61012002F04FFF81B2B1FBF8F7A2
:10D140004FF4FA71012002F047FF81B2B1FBF8F011
:10D15000BAF81010B94279D9AAF8107070E1FEF748
:10D16000F1FC01216846FEF79BFC009806B2012005
:10D1700001F0C8FFF948007890B1FEF77FFC07B2D4
:10D18000BDB13146012002F027FF06B207F132009F
:10D1900086420ADA6438864207DD97FBF8F206E039
:10D1A000FEF754FCFEF764FDE9E796FBF8F2ECA10C
:10D1B0000CE007F11200864205DA2438864202DDCF
:10D1C00097FBF8F201E096FBF8F2E7A102A803F062
:10D1D0005FFA42F22830864204DA022102AA0846A7
:10D1E000FDF7DEFADD48007820B1FEF747FC064681
:10D1F000DFA20CE0FEF72AFCFEF73AFD0646FEF73A
:10D2000025FC421CDBA102A803F042FA02AA182165
:10D210005620FDF7EDFA474601E0FDE0FFE0B6FBE2
:10D22000F7F2D5A102A803F033FA02AA1021642074
:10D23000FDF7FEFA9AF80200564640B1401EB07063
:10D24000CEA210215820FDF7D3FA08E0F4E008231D
:10D25000062210215820CDF80090FCF7B9F9F069AA
:10D260004FF00001002868462CD0FEF719FCF06949
:10D270000099B0FBF7F2801A89B20844F061B0FB64
:10D28000F7F04FF47A7100F5FA70B0FBF1F2BCA13F
:10D2900002A803F0FDF902AA00216420FDF7A8FA14
:10D2A000707830B186F8019001F06CF8F08201F0EE
:10D2B0007DF8042C0ED0052C24D0012C48D0022C53
:10D2C0005DD092E0FEF7ECFB009880B200EB8000AE
:10D2D0004000D3E7FEF7BAFBFEF7CAFCB0FBF7F05D
:10D2E00030820020FCF77EF90220FCF7F1F80420E0
:10D2F00001F00EFF012341F2883206210DA802F051
:10D300001FF872E0002001F0FDFE0020FCF76AF932
:10D31000002001F0FDFE0220FCF7DAF8002213469F
:10D320000C2001F00FFF012001F0C8FBFCF76AF8A8
:10D3300080B2FBF7AFF802460B46002001F002FF77
:10D340003220FDF7D1F8FEF72DFB86F803B04CE054
:10D35000FEF77CFB401C07B2022F00DD0027B8B2AD
:10D3600001F0DEFEB8B2FEF783FC00B225B1014643
:10D37000002002F031FE00B201F0B6FE35E0F07A96
:10D3800088B116216846FEF78BFB009D86F80B904E
:10D3900006216846FEF784FB0098FBF7A1F830836E
:10D3A00028B201F0A1FE708B401C80B270830F2860
:10D3B0001BD3A6F81A90717B484649B17249CDE952
:10D3C000001010230C220021562002F035F906E04F
:10D3D000009010230C2200215620FCF7F9F800F0F1
:10D3E0008DFC707B28B100207073FEF783F910B1BB
:10D3F00011E00120F8E7F07A68B986F80BB0308BBD
:10D4000000B201F071FE10230C2200215620CDF84D
:10D410000090FCF7DDF8347311B0BDE8F08FBAF876
:10D4200010004FF4C872904202D9AAF8102007E009
:10D43000322805D2322001E0814201D2AAF8100040
:10D4400052A200211C20FDF7F3F95746BAF810202C
:10D4500049A102A803F01CF902AA10213220FDF70D
:10D46000E7F910231A4619460220CDF80090FDF77F
:10D4700081F910231A4619467020CDF800B0FDF747
:10D4800079F900F03BFC4FF6FF78042C08D0052C0E
:10D4900006D0012C07D0022C05D0072C0ED02FE08F
:10D4A000388A304401E0388A801B3882012341F2F7
:10D4B000883206210DA801F043FF21E03C8A0020BC
:10D4C000FCF790F825B12146002002F085FD84B2DA
:10D4D00004EB8400400000B201F006FEFEF7B6FA4D
:10D4E000398A01EB810208EA420101F06DFF012057
:10D4F000FBF7EEFF032001F00BFE002001F002FE1F
:10D500009DF82900002887D0388A464600EB800025
:10D5100008EA400425B12146002002F05DFD84B2F6
:10D520000020FCF75FF820B201F0DEFDFEF78EFA76
:10D53000398A01EB810106EA410101F045FF012032
:10D54000FBF7C6FF032001F0E3FD0620FCF752F8CD
:10D55000002001F0D7FD5FE79C0100204901002079
:10D560002533643C000000002533643B00000000CC
:10D570007A5A000054256400253364004D000000F1
:10D5800025326456000000009C300108576F726B12
:10D590002054656D7000000008B50121042001F0E1
:10D5A000EDF84FF4A060ADF8000048208DF80300BE
:10D5B00003208DF8020069460148FDF72BFF08BDE6
:10D5C000000801402DE9F0474B49D1F820014B4DAF
:10D5D0002A6840EA42002860D1F828116A684FF0B2
:10D5E000000A41EA4201A5F108076960401C01D127
:10D5F00087F802A0414E00244FF00109361F4FF07A
:10D60000FF3855F82400FEF77BF83055F87858B10C
:10D610002878C00708D02879C00705D087F803A06C
:10D62000C5F80080C5F804803078022813D97078D6
:10D63000022810D92878C0070DD02879C0070AD051
:10D640000720FEF707FFC5F80080C5F8048086F8BC
:10D6500000A086F801A0305D20282FD3F87810BBF9
:10D6600014B1012C12D01FE0307820281FD370781D
:10D6700005281FD80220FEF7EDFE787808B987F854
:10D680000390B87878B987F802902FE07078202856
:10D690000AD33078052807D80520FEF7DBFE787816
:10D6A00008B987F8039021E03078202802D27078FA
:10D6B00020281BD30820FEF7CDFEF2E7B0B115F805
:10D6C0002400C00712D01CB12868401C09D00DE00E
:10D6D0006868401C0AD10120FEF7BCFEC5F8008036
:10D6E00004E00420FEF7B6FEC5F80480641CE4B232
:10D6F000022C86D3BDE8F0870000214210000020F4
:10D70000164A10B5126800212128137803F07F0310
:10D7100002D0202804D009E0212B1DD1104914E0AB
:10D72000212B00D10F49104C20232370137803F0D4
:10D730007F03212B09D1FE2807D1508828B9908872
:10D7400018B9D088012800D1084929B10020916179
:10D7500050828847002010BD022010BD1403002015
:10D760000D960008299600083002002095BC00089C
:10D77000014902F0F1B9000048020020014902F01D
:10D78000EBB900004002002005490968C978052965
:10D7900001D900207047034A02EBC10102F0DCB955
:10D7A000140300208002002009B9002800D00220C4
:10D7B00070470000124910B509680A7802F07F022C
:10D7C000212A0CD1FF2804D0022816D0222814D0F8
:10D7D00005E0488818B9888808B9C88808B10220C7
:10D7E00010BD0120FBF7A4FE0220FBF78DFE0649C9
:10D7F00004480860054900200870002010BD0000A2
:10D800001403002055534243A8340020CC010020CB
:10D8100070B54C4800254D4985724B480968C07960
:10D820004872284601F08AFB4FF40071002001F095
:10D8300041FC2021002001F025FC4021002001F0C6
:10D84000A9FB434C002014F82C1F01F0B3FB8021EE
:10D85000002001F0F9FB0020FBF798FE002001F00A
:10D86000E1FB0021012001F025FCC021012001F095
:10D87000EBFB2021012001F005FC0021012001F03B
:10D88000B9FB0021022001F015FC4FF48071022049
:10D8900001F080FB2178022001F08CFB4FF4405610
:10D8A0003146022001F0A6FB0021022001F0EAFB34
:10D8B0000021032001F0FEFB4FF4A071032001F0D2
:10D8C000C3FB2021032001F0DDFB0021032001F038
:10D8D00091FBF110042001F0EDFB7111042001F027
:10D8E000B3FB0021042001F085FB2021042001F07E
:10D8F000C9FB0021052001F0DDFB4FF4C8710520B4
:10D9000001F048FB4021052001F054FB3146052081
:10D9100001F070FB0021052001F0B4FB217800200C
:10D9200001F048FB002001F07DFB002001F00EFB20
:10D93000084901200860094907480860084805703F
:10D9400070BD000018350020CE30010814030020FF
:10D9500050020020D002002055534243A83400203A
:10D96000CC01002003480178202901D10021017059
:10D97000704700003002002070470000094810B5D1
:10D9800000680024847200F0EBFC0748046007493B
:10D990004FF4044008800449091F086004480460EB
:10D9A00010BD000014030020445C00402003002050
:10D9B000D0020020044805490068884202D00220B5
:10D9C000FBF7B8BA70470000A83400205553424313
:10D9D000124A10B5107802280AD04FF44054032898
:10D9E00010D0042801D0052816D1002010700DE0B9
:10D9F0000B48C07B28280FD1D2E90101BDE81040B7
:10DA000001F000B90121002001F0FEFC2146BDE833
:10DA10001040022001F0EEBA10BD0000CC01002041
:10DA2000A834002070B51648C47B0220FDF7F0FE34
:10DA3000144D02464FF4807168801148403800F060
:10DA40004BFB287818B1012805D0022006E0BDE87C
:10DA50007040FBF78FBA2A2C0CD00120FBF76AFA32
:10DA60002421052001F0F4FCBDE8704000210220D3
:10DA700001F0CABCD5E90101BDE8704001F042B92E
:10DA8000A8340020CC010020094810B50068807A35
:10DA900000280BD00749052008600120FBF748FD4E
:10DAA0000220FBF731FD04490020087010BD000082
:10DAB00014030020D0020020CC01002001490420E2
:10DAC00008607047D0020020FEE700002DE9F04119
:10DAD00001880B0401F01F0249D4284B11F4E04FD8
:10DAE00003F108044FF0050C21784FF004064FF0C5
:10DAF00001054FF0020706D0012A31D00A2A16D0BC
:10DB00000F2A38D130E0012A04D0042A04D0062A92
:10DB100031D104E05F702EE083F801C02BE05E702D
:10DB2000022914D0072912D0052910D023E04288F9
:10DB3000808802EB00400322B7EB106F01D1DA704E
:10DB400019E0B2EB106F04D1DE70032913D16580A8
:10DB500011E0B6EB106F0ED1678083F803C00AE0C6
:10DB600000F018FA2570F2E702F036FC03E0112A03
:10DB700001D1FCF7DFFF0020BDE8F081C0010020EB
:10DB80007047704710B501464FF0006000F042F852
:10DB9000BDE810404FF4A06000F032B830B50F235C
:10DBA000C27801780125F2B1144A126801F1E0212E
:10DBB00002F4E062C2F5E062120AC2F10404D3404A
:10DBC0004278A24084781C401443220181F800244A
:10DBD000007800F01F018D404009800000F1E02036
:10DBE000C0F8005130BD01F01F0085404809800099
:10DBF00000F1E020C0F8805130BD00000CED00E0E5
:10DC00000249084302490860704700000000FA0515
:10DC10000CED00E0024A11400143024801607047E8
:10DC200080FFFF1F08ED00E070B52F4D29680878D0
:10DC30004C78420606D000F07F00012828D0022848
:10DC40002BD035E0092C06D0052C07D0032C0ED0A4
:10DC5000012C14D02CE001F0EBFF28E0C8787F28DD
:10DC60002ED8887860BB888850BB887A27E0C8782F
:10DC700001281DD18888D8B901F0F6FF17E0C878CF
:10DC8000012815D1888898B9487A80060AD40FE00F
:10DC90000B2C0DD102F03EF809E0012C02D0032C30
:10DCA00003D005E001F0C6FE01E001F0EFFF58B13E
:10DCB0000E492046096849698847032802D018B1EF
:10DCC00008200DE009200BE0094A06200021126817
:10DCD000084B120403EBD2325160074A3021118005
:10DCE0002968087270BD000014030020180300208A
:10DCF000505C004000600040240300201CB500215F
:10DD00000448CDE9000120238022084600F03EF8B7
:10DD100000201CBD4C3100200A2805D800EB8000F3
:10DD20008006000E00F026B87047000010B50028ED
:10DD30001DDB00291BDB802819DC202917DCCB1711
:10DD400001EB5373C3F3C70423F00703C91A01237C
:10DD50008B4000EBC410D9B2B0F5007F07DC044B58
:10DD6000002A1A5C01D00A4300E08A431A5410BD0D
:10DD70004C31002010B504463C218120FEF71CF9EF
:10DD80002046BDE810403C21FEF716B92DE9F843C6
:10DD90000546DDE90879C8189046C0B24B074FF038
:10DDA000010206D002EBD104410704D002EBD006F9
:10DDB0001FE0CC08F8E7C6081BE004F1B000C0B2D1
:10DDC0003C21FEF7F9F8102040EA15103C21FEF73F
:10DDD000F3F805F00F003C21FEF7EEF801233C229A
:10DDE00041463846CDF80090FEF7F9F8641C4744E8
:10DDF000E4B2B442E1D33846BDE8F88310B50F4C25
:10DE00002068007A022811D004280FD0032804D0FB
:10DE1000052802D0072805D008E0FCF735FA20686D
:10DE2000007A04E006480068C0688047082021683E
:10DE30000872BDE8104000F05BBA00001403002037
:10DE400018030020F0B5DFF854E00025BEF808C044
:10DE500020E00EEB0514267B9E4219D1012E02D044
:10DE6000022E15D107E0D4E904648EB186420FD1A9
:10DE70008C4209D20CE0D4E90476A469874207D326
:10DE8000864205D8A14203D86D1C15800020F0BD44
:10DE90006D1CEDB26545DCD30320F0BDA43300203A
:10DEA0002DE9F047394B002103F10802D8880227F9
:10DEB0000A3084B2DC80104692F800C00125344E4E
:10DEC00040884FF00709BCF1080F5CD2DFE80CF086
:10DED0005B040F38464E552B10B1012804D052E098
:10DEE0000720FBF7E3FF4EE0518017703BE001286D
:10DEF00002D0022814D046E05180D878012805D0FD
:10DF00003078022807D0012808D03CE003201070A8
:10DF1000FCF7B0FD37E082F800902CE0082029E003
:10DF2000518015702FE040F6B83084422BD318484A
:10DF3000D980AC30D0E901120220FDF77FF822E051
:10DF4000012802D0022804D01DE051800420107066
:10DF500019E0518082F80090377014E0012812D146
:10DF6000518005201070FDF759F90CE001280AD105
:10DF70005180062010709D7005E0B4F5967F02D3A5
:10DF8000D980FCF73FFD0020BDE8F087C0010020EC
:10DF9000A43300202DE9F047C2B005460024AC218F
:10DFA0006846FAF7D4F82888ADF8B0002888002130
:10DFB000C0F30230ADF8AC00DFF814A101266F46C3
:10DFC0004FF002098C4623E005EB8100D0F80220D7
:10DFD0002BA800EBC100C260083041B9130206D57E
:10DFE0009AF80380B8F1000F01D18AF80360930F0B
:10DFF00025D00323B3EB927F06D112F0405F48D0C7
:10E00000C2F30172012A44D080F800C0491CC9B291
:10E01000BDF8AC008842D7D89DF8AE008DF800005E
:10E02000AC2239462B48FAF779F82A4858222BA90E
:10E030005838FAF773F842B00020BDE8F087067050
:10E040009DF8AE200AB98DF8AE6007EB01124FF0D3
:10E05000320816734368C3F3892000FB08F0C3F34A
:10E06000090303EB83084FEA4808C2E904084FF4A8
:10E070007A72B0FBF2F0584300EB80004000A042FF
:10E0800001D904460190BDF80800401CADF8080015
:10E09000BCE780F800909DF8AE204B46032A01D0E3
:10E0A0008DF8AE3007EB01124FF06408137340682F
:10E0B000C0F3072303FB08F35361C0F3474303FB9B
:10E0C00008F3136100F07F00322358439061DAE7D0
:10E0D000C0010020A4330020064B521C520803EB61
:10E0E000410105D031F8043B20F8023B521EF9D122
:10E0F0007047000000600040704700001CB50B2115
:10E100006846FDF7CDFC0848002101604160816050
:10E11000C1600162016105494161054981614FF0BA
:10E120007E51C1611CBD00003803002000007A430D
:10E13000333333402DE9F05F4FF000090126DFF85B
:10E140008C81634DB346CA46FAF785F96860044688
:10E150002F6821463846FAF78AF8A8605D493846A4
:10E16000FAF733F82146FAF737FA04D298F808108C
:10E17000491C88F8081098F8080047464FF0000836
:10E180000A2801D9C5F8208053492868FAF71DF8F4
:10E190006968FAF721FA01D287F80880D5E90010FA
:10E1A000FAF71AFA01D287F808804C48A968814228
:10E1B0000CDA387A4FF0010918B9286AFAF705F82D
:10E1C00028624748296A814200DD2862D5E90001BA
:10E1D000FAF702FA0CD2D5E90010FAF748F8FAF784
:10E1E00066F900B2322803DD4FF00009C5F820803F
:10E1F0003C49AC688C4203DC3B48844200D8002692
:10E200003848844207DD2046E968FAF730F810F113
:10E21000FF4F00D300263448844207D92046E968DE
:10E22000FAF725F8B0F5000F00DB00262D488442F0
:10E2300006DC2D48844203D8DFF8B0A04FF0000B75
:10E240005846FAF711F9834621466869FAF715F836
:10E250005946FAF712F8834678624846FAF704F905
:10E2600081465146A869FAF702F84946FAF705F8D7
:10E27000296AFAF702F88146B8623046FAF7F4F8EC
:10E2800006462046E968F9F7F2FFE969F9F7F5FF74
:10E290003146F9F7F2FF0646F86249465846F9F763
:10E2A00094FF3146F9F791FFFAF701F9C5E9034008
:10E2B000002802DCC5F8108004E041F28831884271
:10E2C00000DD2961288A80B2BDE8F09F1C00002093
:10E2D000380300200000F0410000F04200004844F4
:10E2E0000050434700008C4200008CC200002040D8
:10E2F0000C4810B590F82C10002000F05BFE0A4886
:10E300000068007A082802D0092809D006E00749E9
:10E310004FF480500880064910200880002010BD6E
:10E32000012010BD50020020140300202203002011
:10E330002403002010B50220FDF77AF904460620D8
:10E34000FDF776F90549844201D9012000E0022059
:10E350000870BDE81040C0B200F092B96000002023
:10E360000648012101600021054A0160031D196072
:10E370004FF4E0511180016000207047405C004084
:10E380002003002008496422C86950430A22B0FBD8
:10E39000F2F00A6AB0FBF2F0002280B2CA610A62AF
:10E3A000642800D9642070471C0000202DE9FC4F30
:10E3B000062618250446642800D9642400213C4818
:10E3C000CDE90001082346221821062001F034F986
:10E3D00004EB441040006421B0FBF1F087B24FF031
:10E3E00008094FF0090A4FF01C0B4FF01D08022FCF
:10E3F00046D9B81E84B2012241464846FFF796FC32
:10E4000001224146D1465046FFF790FC0122D846F2
:10E4100059464846FFF78AFC412F2DD3641E4FF022
:10E420001B0A4FF04809A4B2012251464846FFF7A3
:10E430007DFC012241464846FFF778FC422F1BD164
:10E44000641EA4B2012251464920FFF76FFC13E07D
:10E450003019C01C07B20122E91C3846FFF766FCE0
:10E4600038460122291DFFF761FC38460122691D4B
:10E47000FFF75CFC641EA4B2002CE9D1BDE8FC8F60
:10E48000012F0CD0022FF9D10122414654465046AB
:10E49000FFF74CFC012259462046FFF747FC02B02B
:10E4A00041464846BDE8F04F0122FFF73FBC00005F
:10E4B000563001082DE9F04FADB00746FDF7D2FA0E
:10E4C000814611216846FDF7EBFA0098FF2580B2DE
:10E4D0004FF4FA681FFA89F1FAF7BCFF4249064681
:10E4E0004FF0020A0878022802D0012879D079E09A
:10E4F000487848B1002048706846FCF799FDAC2286
:10E5000069463A48F9F70AFEDFF8E0B09BF80000E8
:10E5100020B1022F06D0012F46D049E001202DB0B6
:10E52000BDE8F08F3149A0220C316846CDF8A090AB
:10E530002C91F9F7F3FDDBE9012329A8DBF80010A2
:10E54000FDF794F8DDE92947CDE92869A02268465E
:10E550002C99F9F7E3FDDBE901232AA8DBF8001089
:10E56000FDF774F9DDE92A01A04203D904460F46FC
:10E570004FF0010A1EB1B44201D9344600E0BCB1EB
:10E5800000263A4621465046FCF758FD05000FD0BC
:10E59000032D0DD0042DC2D1761CB6B23220FBF76C
:10E5A000A3FF032EEDD91DE0FCF738FE41F28834BD
:10E5B000FDF7C8FA04EB080700F52F76FCF732FDEB
:10E5C000042806D00125FDF7BDFAB042F6D909E0CE
:10E5D00007E0FAF717FFA4EB08018142F3D2874264
:10E5E000F1D9002528469AE760000020D4030020D6
:10E5F0001CB509216846FDF753FA0098112184B231
:10E600006846FDF74DFA0A216846FDF749FA009879
:10E610001649C0B20228887002D10870FAF740FF8C
:10E6200001F064FDE0B2FFF777FB0020FAF7DAFFB4
:10E630000FA208211420FCF7FBF80FA208214420A8
:10E64000FCF7F6F8FFF75AFBFFF774FE00221346BB
:10E650000C2000F077FDFDF73DFC002000F058FD98
:10E66000FAF744FEBDE81C40FFF748BD4801002012
:10E67000545331303100000056322E30310000004A
:10E6800070B5114D114E4FF4004401280CD00228F2
:10E690004FF0100130460ED0FCF73DFF21462846D2
:10E6A000BDE87040FCF737BF21462846FCF733FF32
:10E6B0001021304603E0FCF72EFF21462846BDE836
:10E6C0007040FCF72ABF000000080140000C014028
:10E6D000F8B501210C2000F051F84FF40044ADF8DA
:10E6E000004010258DF8035003200B4E8DF80200DA
:10E6F00069463046FCF78EFEADF80050074D69467E
:10E700002846FCF787FE21463046FCF704FF10211F
:10E710002846FCF700FFF8BD00080140000C01404E
:10E7200010B5292208490948F9F7F8FC064991F87B
:10E730002920064880F82920C96AC1620249183890
:10E740002039096D816410BD68010020E43000208B
:10E75000034A516821F44041014351607047000071
:10E7600000100240044A0029D16901D0014300E0B1
:10E770008143D1617047000000100240044A002923
:10E78000916901D0014300E081439161704700002D
:10E7900000100240044A0029D16801D0014300E082
:10E7A0008143D16070470000001002401B4810B543
:10E7B000016841F010010160016821F0030101606E
:10E7C000016841F00201016000F02AF8012000F028
:10E7D00071F8212000F044F80028FAD0002000F061
:10E7E0005FF84FF4806000F06BF8002000F072F8E2
:10E7F0004FF42011002000F07DF8012000F074F8A3
:10E80000392000F02DF80028FAD0022000F07CF822
:10E8100000F03EF80828FBD110BD000000200240A7
:10E820000C48016841F00101016041680A4A114049
:10E8300041600168094A11400160016821F48021AA
:10E840000160416821F4FE0141604FF41F018160C5
:10E8500070470000001002400000FFF8FFFFF6FEC6
:10E86000034600205909094A01290AD002290AD081
:10E87000516A03F01F02012393400B4200D0012094
:10E8800070471168F5E7116AF3E7000000100240D5
:10E890000248406800F00C00704700000010024081
:10E8A000034A516821F0F0010143516070470000B4
:10E8B0000010024001490860704700000000424219
:10E8C000034A516821F4E061014351607047000040
:10E8D00000100240034A516821F4605141EAC0002F
:10E8E0005060704700100240014908667047000000
:10E8F00000004242034B5A68084322F47C12104342
:10E900005860704700100240034A516821F003012B
:10E910000143516070470000001002400149C1F8F6
:10E92000D80070470000424238B501210420FFF7AB
:10E9300025FF0220ADF8000010208DF80300032011
:10E94000054C8DF8020069462046FCF763FD022164
:10E950002046FCF7E0FD38BD000801402DE9F041FC
:10E96000FCF742FB14480024015DF1B10021134F74
:10E97000015507EB8420FCF7BBFA1148002500EB9A
:10E9800084264FF4806805EB842036F8021B384457
:10E99000FCF7FCFA042804D0FCF7F0FA0420BDE8E8
:10E9A000F081AD1C4545EED302E0641C102CDBD396
:10E9B000FCF7E4FA0020F2E7802E00200090010826
:10E9C000800400202DE9F041104DFCF70DFB104EA6
:10E9D000002406EB8420FCF78BFA641CA4B2092CFB
:10E9E000F7D300244FF4185735F8021BA019FCF791
:10E9F000CDFA042802D00420BDE8F081A41CA4B202
:10EA0000BC42F1D3FCF7BAFA0020F5E780040020FD
:10EA10000090010810B5264CA268137813B1012BA1
:10EA200006D028E040022061480260610120107099
:10EA30006068806960B3A169E06840220844C02131
:10EA400001F0B6FC6068816940398161A06940309D
:10EA5000A0614021012000F007FB3021012000F0DF
:10EA600011FB2069403020616069403860611148C5
:10EA70008168403981606069002808D161680E4A68
:10EA80008861A061032120611170A168087010BD28
:10EA9000D4E90301FBF762FD4022C021E06801F0E8
:10EAA00087FC61684FF4E07088614020D0E7000087
:10EAB00064000020C8340020CC01002070B5054659
:10EAC000002401F045FD2846FFF7F4FC002803D0A0
:10EAD000641CE4B2022CF4D370BD10B540F6B8311A
:10EAE000818040F6E441C18040F6AC53038140F69A
:10EAF000C4114181B4214182F0218182032202822A
:10EB00000121C1820021018340F6D864C48341837E
:10EB100083830A23038481844184C28410BD10B599
:10EB2000002000F0F5FA0220FAF7D2FC002213468A
:10EB30000C2000F007FBBDE810400120FFF7BEBF2E
:10EB400010B51144B1F5805F09D92A2802D10220FD
:10EB5000FAF7F0F90020FAF7EDF921210AE00C4963
:10EB60008968B1EB422F10D02A280CD00020FAF788
:10EB7000E1F92421052000F06BFC0021012000F0C8
:10EB800043FC002010BD0220F1E7012010BD000071
:10EB9000A83400200649087CC00702D0054805219A
:10EBA00004E0C97C0448242900D9242101F0BEBA1C
:10EBB000A8340020D80200209E3101080A4810B570
:10EBC000816811B1007B000601D5002000E0022021
:10EBD000FAF7B0F92021052000F03AFC0021BDE849
:10EBE0001040012000F010BCA8340020082101488A
:10EBF00001F09CBADD0200200421014801F096BA20
:10EC0000D402002070B5154C0D460646217831B16E
:10EC1000022921D12946BDE87040FFF7FBBE01461D
:10EC20002A462820FFF78CFF002815D00C48007BCF
:10EC300000064FF0020003D5207029463046EAE76F
:10EC4000FAF778F92421052000F002FCBDE87040B5
:10EC50000121084600F0D8BB70BD0000CC010020A7
:10EC6000A8340020074800210F22017041708270F3
:10EC7000FF22C2700171417102228271C1710821AB
:10EC800001F054BAE5020020064800210222017179
:10EC900041718271C17141728272C1720C2101F0A5
:10ECA00045BA0000FF0200200348C17C122900D9A8
:10ECB0001221024801F03ABAA8340020ED020020E7
:10ECC0000121002000F0A0BB0121002000F09CBB2E
:10ECD0000B4810B5816829B9007C400702D4012196
:10ECE000002008E00220FAF725F92421052000F091
:10ECF000AFFB00210120BDE8104000F085BB000003
:10ED0000A834002010B5164C0A46217831B10129EB
:10ED100024D1BDE81040114601F064BC01462A2010
:10ED2000FFF70EFF002819D00E48007B000608D41C
:10ED300001202070BDE810404FF44051022000F047
:10ED400059B90020FAF7F6F82421052000F080FBDD
:10ED50000021BDE81040012000F056BB10BD0000AE
:10ED6000CC010020A83400207047000010B5084CEA
:10ED70000648082120604FF4C87060602046FAF70A
:10ED8000BFF9A060BDE8104000F088B855AA5AA5A8
:10ED90005400002002490A6A1044086270470000CB
:10EDA0001C0000200249CA691044C8617047000075
:10EDB0001C00002010B5044602EB82004FF6FF73E2
:10EDC000C91F03EA400010290AD2DFE801F0080A4F
:10EDD0000C5D0E1214162D1C1057595F5B61A0803C
:10EDE00010BDE08010BD208110BD608110BDE083AA
:10EDF00010BD628210BDA28210BD2282BDE810400B
:10EE0000D0B2FEF789BF2348E282022A027022486C
:10EE100006D0012101700846BDE81040FAF740BB5A
:10EE2000022101700846F7E7208B9042E4D022834C
:10EE3000A18882B1012001F0CFF8A080E1880120F3
:10EE400001F0CAF8E0802189012001F0C5F8208195
:10EE5000618901200FE0002001F0BEF8A080E18868
:10EE6000002001F0B9F8E0802189002001F0B4F819
:10EE700020816189002001F0AFF8B6E7628310BD00
:10EE8000A28310BDA28410BD228410BD628410BD77
:10EE9000E28410BD4A0100204801002070B50B4DEE
:10EEA00000240C220A492846FCF70EFA38B1641CEB
:10EEB000E4B21420FBF718FB032CF2D301E0032C7F
:10EEC00001D3012070BD002070BD000000F00108DA
:10EED000540000202DE9FF41164C0E460746002540
:10EEE00020680090606801902089ADF80800A07A41
:10EEF0008DF80A000B21684601F010FA0B22394602
:10EF00006846F9F74CF940B16D1CADB22034102DB4
:10EF1000E6D3002004B0BDE8F081A08B3080608B88
:10EF2000ADF80C000448BDF80C1000EB412000F5D2
:10EF30000070EFE78008002080040020024920F0E4
:10EF40000700086070470000505C0040F0B50E49B3
:10EF50000E4E48F68F770D78002148F2800C0BE0BA
:10EF6000CAB206EB8203D3F8004C3C40144344EA97
:10EF70000C04C3F8004C491CA942F1D3044940F0E9
:10EF800080000860F0BD0000A80200200050004092
:10EF90004C5C0040054A21F00101126892B202EB7C
:10EFA000C000034A02EB400081607047505C0040A3
:10EFB000006000400D4A12683E2992B202EBC00088
:10EFC0000B4A02EB400209D94809C90601D1401E8B
:10EFD00080B24FF4004141EA802004E04808C907AC
:10EFE00000D0401C8002106070470000505C004060
:10EFF0000C60004082000A480244D2F8000C4BF634
:10F000008F731840CB0401D580F48050890401D55A
:10F0100080F4005048F280010843C2F8000C7047A9
:10F0200000500040810007480844D0F8001C4BF60F
:10F030008F72114081F4405148F280021143C0F8B0
:10F04000001C704700500040054A21F00101126881
:10F0500092B202EBC000034A42F810107047000061
:10F06000505C004000600040044A126892B202EB1B
:10F07000C000034A02EB400041607047505C004012
:10F080000060004082000A480244D2F8000C48F6B2
:10F09000BF731840CB0601D580F01000890601D55A
:10F0A00080F0200048F280010843C2F8000C70474D
:10F0B00000500040820005481044D0F8002C48F66B
:10F0C0008F131A400A43C0F8002C704700500040CC
:10F0D0000149C870704700001C00002001490882E7
:10F0E000704700001C00002010B5A0F5FA7140F632
:10F0F000AD52914203D2F9F7AEF90149086010BD53
:10F1000038030020014948707047000008000020C3
:10F11000192801D20149C873704700009C010020E2
:10F1200001494882704700004801002001494870A9
:10F13000704700009C0100200149C8707047000022
:10F140004801002070B5182819D20E2817D05F4C3E
:10F150004FF46B75182812D2DFE800F00C12181E5D
:10F16000242A114F5A656E30363D11787F8E85AC5A
:10F17000949AA0B210461946F9F7E5F9208070BDBF
:10F1800010461946F9F7C0F9608070BD104619465F
:10F19000F9F7D9F9A08070BD10461946F9F7D3F9EF
:10F1A000E08070BD10461946F9F7CDF9208170BD99
:10F1B00010461946F9F7C7F9608170BD1046194627
:10F1C000F9F7EDF9E06070BD10461946F9F7BBF9A3
:10F1D00084F8290070BD10461946F9F7B4F90028E3
:10F1E000F8D0092803D2E16A0843E06270BDE16A01
:10F1F00020F040408143E16270BD10461946F9F7A6
:10F20000A2F980B2A0F13C01A942F5D2608270BDA2
:10F2100010461946F9F797F980B2A0F13C01A942CE
:10F22000F5D2A08270BD10461946F9F78CF980B26C
:10F23000411E0A29F6D207E010461946F9F783F96C
:10F2400080B2411E0229EDD2208270BD10461946BF
:10F25000F9F779F984F8280070BD10461946F9F7D6
:10F2600072F9208370BD10461946F9F76CF980B227
:10F270000128F7D8608470BD10461946F9F763F984
:10F28000A08470BD10461946F9F75DF9608370BD22
:10F2900010461946F9F757F9A08370BD1046194674
:10F2A000F9F751F980B2A0F13201B1F5AF7FF4D88E
:10F2B000E08370BD10461946F9F745F9208470BD0A
:10F2C00010461946F9F73FF9E08470BDE43000209C
:10F2D0007CB578B1012830D110216846FCF7E0FBFD
:10F2E000009805B21548408A48B1012809D0022883
:10F2F0000DD120E0BDE87C400220FAF7E9B80221F8
:10F3000000E003216846FCF7CBFB009884B225B1EE
:10F310002146002000F060FE84B220B2FFF7E4FE38
:10F320000120FAF7D5F8FCF797FB012805D1BDE8D5
:10F330007C40FAF7C3BE0421E4E77CBD480100200D
:10F340002DE9F0410026984615460F4604460A2945
:10F350000CD3307820707078607002200168C4F897
:10F3600002104168C4F8061000891BE0FCF7EAFBB4
:10F370000E4B421907EB470103EB810042604670D8
:10F38000A0F80280012203F82120856022704178D4
:10F390006170D0F80210C4F80210D0F80610C4F85A
:10F3A000061040896081BDE8F08100005C03002008
:10F3B00010B5044C082160602046F9F7A1FEA0605A
:10F3C000002010BD5400002010B568B1012812D0F3
:10F3D000022817D10846F9F75DF802460B460420CB
:10F3E000BDE81040FFF7AEBE0846F9F753F80246F5
:10F3F0000B460220F4E70846F9F74CF802460B46A4
:10F400000320EDE710BD000010B50F4A0C460D4972
:10F41000116010730D22C0210B4800F0C9FF0D21AF
:10F420000120FFF721FE09480521002C017007D0BB
:10F43000042101703021BDE810400120FFF722BEF9
:10F4400010BD000055534253C8340020CC010020A9
:10F45000014A907011737047ED02002000B589B029
:10F4600020220A496846F8F759FE094800216A46F1
:10F4700052F8213040F82130491C0829F8D30922DC
:10F4800004A1F8F74BFE09B000BD00004C220108B2
:10F49000A008002054533130315F4150500000002B
:10F4A00070B516480068174D0004C10B144801449C
:10F4B000098989B200EB41042868017A09290FD033
:10F4C0002178017061784170A088F9F74DFD2968B5
:10F4D00048802089F9F748FD29688880A089C8807C
:10F4E000286801210172C08828B1FAF71FFFBDE822
:10F4F0007040FEF7FDBEFEF797FBF8E7505C00405A
:10F5000000600040140300202DE9F04387B08146DD
:10F5100001216846FCF7C4FA009804B2FCF71EFB10
:10F5200005460A216846FCF7BBFA0098DFF800811F
:10F5300086B200279DB3FCF70BFB012830D1B4F550
:10F54000C87F2DDD10216846FCF7AAFA0098CDE9A6
:10F55000008785B2102330220821184600F06CF88D
:10F5600008F5C070CDE900071023302208214020A3
:10F5700000F062F825B12146012000F02DFD04B213
:10F580000A2094FBF0F22BA102A801F081F802AA54
:10F590000E215620FBF72CF907B0BDE8F083FFE7FA
:10F5A000002010254024022E02D1032040251024E3
:10F5B0001F4E5FEA090106F1600619D0012926D025
:10F5C000022915D0B9F1030FE6D11023302208210A
:10F5D0002046CDE9006700F02FF806F1C000CDE924
:10F5E0000007102330220821284600F025F8D3E731
:10F5F000CDE90080102330220821284600F01CF8B5
:10F600001023302208212046CDE90067EDE7CDE93F
:10F610000080102330220821284600F00DF804480D
:10F620001023C030CDE90007302208212046DCE756
:10F63000762E0108253364002DE9FF4F84B006467D
:10F64000009007980C460F46401EC11700EB517002
:10F650000121924601EBE00000FB0AF0039006EB6B
:10F660000A0080B2DDF844B04FF000080190404637
:10F670000399029088425ED2129828B101280FD0D7
:10F68000022822D0032822D1E01BC11700EB5170C1
:10F69000C11001FB0A610098091A11F80B5016E01D
:10F6A000E01BC11700EB5170C11001FB0A6100980B
:10F6B000091AE01711F80B5004EB5070C0101F49E5
:10F6C00006EBC010405C054301E00BF0FF054FF076
:10F6D0000009129803284FEAC57006D008B101222C
:10F6E00000E000222146304609E000280198A0EB06
:10F6F000080000B201D0012200E000222146FEF7FE
:10F7000015FB641C24B207986D08E11B814207D1E8
:10F71000761C08F101003C4636B21FFA80F806E07C
:10F7200009F101001FFA80F9B9F1080FD1D302984D
:10F73000401C80B29CE708B0BDE8F08F4C3100203F
:10F7400008B50028009001D0401EFAE708BD00006F
:10F7500008B501210820FFF711F80320ADF80000DB
:10F7600014218DF803108DF8020069460148FBF75B
:10F7700051FE08BD000C014010B500240123094AC8
:10F78000012805D0022802D149B1C2F8843110BD48
:10F7900011B1C2F8803110BDC2F8804110BDC2F86D
:10F7A000844110BD0080214270B50A4C0025C4F888
:10F7B00080510120C4F88401C4F88001284604F572
:10F7C000C074FFF7BDFF65600020FFF7B9FF25603B
:10F7D00070BD00000080214270B50D4C0025C4F8BA
:10F7E0008051C4F88451284604F5C074FFF7A8FF7F
:10F7F000012626600020FFF7A3FF66600020FFF7C8
:10F800009FFF2560BDE870400020FFF799BF000012
:10F81000008021422DE9F041082407464FF00008FE
:10F8200001261E4D14E000210120FFF7A5FF380638
:10F8300002D5C5F8846101E0C5F884810020FFF796
:10F840007FFFC5F880610020FFF77AFF7806070E7A
:10F85000641EE4B2E7D24746C5F88081C5F88461EA
:10F86000DFF83C80FF240020FFF76AFF02214046BA
:10F87000FBF74AFE30B1641E14F0FF04F3D1002000
:10F88000BDE8F081C5F880610020FFF759FFC5F899
:10F8900080710020FFF754FF0120F1E70080214232
:10F8A000000C01402DE9FC4180460C216846FCF724
:10F8B000F7F80098574EC4B20025B0790227844269
:10F8C00012D0F582012C01D024B106E028B9F571DF
:10F8D000757002E0012800D1F77107216846FCF736
:10F8E000DFF800987083B471F08A401CF082B8F1A0
:10F8F000000F02D1F078022822D1F570F582F0795C
:10F90000012802D003281BD106E0308B00B2FFF79C
:10F91000EBFB7570F5710DE009216846FCF7C0F846
:10F92000002213460C20009CFFF70CFCE0B2FEF70F
:10F93000F3F9F77107216846FCF7B2F80098708375
:10F94000F08A718B88421FD3F079F8B1012846D034
:10F95000022819D101216846FCF7A2F8009800B2EC
:10F96000B0F5C87F10DA00222B4B0C20FFF7EAFB22
:10F970000220F9F7ADFD0020FEF7CEF975700320E7
:10F98000F071F5820120F070BDE8FC81FCF776F89B
:10F99000044610216846FCF783F800984FF00108F0
:10F9A00087B286F8018006216846FCF779F800984E
:10F9B000F8F796FD308327B12146002000F00CFBBC
:10F9C00084B220B2FFF790FB08216846FCF768F884
:10F9D0000098708386F807804046F582D3E70F21B0
:10F9E0006846FCF75DF80020F9F7FCFD0020FFF702
:10F9F0008FFB0220F9F76CFD002213460C20FFF765
:10FA0000A1FB7570F771F582BDE8FC41C820FAF7DB
:10FA10006BBD0000480100200000084000214FF4A9
:10FA20007A720020401C6428FCDB491C9142F8DB00
:10FA3000704700002DE9F04138480068017811F066
:10FA40007F0102D0022905D066E0417A01F0DF0192
:10FA500041724EE0418800295ED10179F1BB4179C4
:10FA6000304D21F080040A0605EB84022C4BD2F8BD
:10FA7000002C03D5C2F30112120102E0C2F30132DD
:10FA800012031E782346A64246D93AB3807A28B399
:10FA900008064FEA84000ED52844D0F8000CC0F3C5
:10FAA0000110012821D11846F9F742FD20463021E6
:10FAB000FFF7E8FA19E04619D6F8000CC0F3013058
:10FAC000012812D14BF68F7748F28008A4B118466E
:10FAD000F9F71AFDD6F8000C384000E01CE080F47D
:10FAE000405040EA0800C6F8000C0F480068406922
:10FAF00080470020BDE8F0810C4890F82C100020D1
:10FB0000FFF758FAD5F8000C384080F4405040EA2E
:10FB10000800C5F8000CE8E70220EBE7140300201A
:10FB2000A8020020005000401C03002050020020CA
:10FB300010B5074C30B1074800680068804720685E
:10FB40000A3010BD216801200882002010BD00008D
:10FB5000140300201C030020054A13685A8A10B1C0
:10FB60000868104470478888801A188200207047FF
:10FB70001403002010B5074C30B1074800688068B6
:10FB8000804720680C3010BD2168012008820020C9
:10FB900010BD0000140300201C030020204910B5F4
:10FBA000096860B11F48002202800A7853060AD013
:10FBB00002F07F02012A16D0022A16D001E00220AC
:10FBC0000882002010BD497A8A06027802D542F0E8
:10FBD000020201E002F0FD0249060270D1B211D426
:10FBE00001F0FE0110E00F4810BD49790A070B062D
:10FBF0000D4901EB9261D1F8001C07D5C1F3011149
:10FC000006E0017841F00101017003E0C1F3013128
:10FC10000129F6D00548006800698047E3E7000045
:10FC2000140300200E030020005000401C0300209D
:10FC30000A4810B500680A4AC1785278914203D840
:10FC400082780AB982880AB1022010BD8172054803
:10FC5000006840688047002010BD000014030020A9
:10FC6000A80200201C030020064810B50068417A55
:10FC700041F02001417204480068C06980470020BB
:10FC800010BD0000140300201C03002070B51D48A7
:10FC90001D4D0268517921F0800005EB80000B06B4
:10FCA000D0F8003C21F0800403D5C3F301131B01FD
:10FCB00002E0C3F301331B03144D2D78A54210D984
:10FCC000548874B96BB1927A5AB10906D0F8001C05
:10FCD00048F2800207D548F6BF73194081F0100141
:10FCE00006E0022070BD4BF68F73194081F48051FD
:10FCF0001143C0F8001C0648006880698047002056
:10FD000070BD00001403002000500040A802002035
:10FD10001C03002010B50E4C0E4A20681268C178F2
:10FD200092694079904721688A7A22B118B9087996
:10FD300008B9887808B1022010BD07480068C0687B
:10FD4000804720684179C172C1780173002010BDDD
:10FD500014030020180300201C03002070B5064681
:10FD6000F8F716FA0004000C23D03418641EB442CD
:10FD700004D3207801F0F6F80028F7D10020607055
:10FD8000354600E06D1C287818B101F0EBF800282A
:10FD9000F8D1AE420DD0611B891C8AB230460021D9
:10FDA00005E015F8013B491C00F8013B89B291427E
:10FDB000F7D3304670BD00007CB50C216846FBF7D8
:10FDC0006FFE00980D21C4B26846FBF769FE009DE6
:10FDD000FBF7E8FD06461648417BA14203D0447379
:10FDE0002046FFF775FAFAF7A3F82DB131462846F9
:10FDF000BDE87C4000F052BB0C216846FBF750FE8A
:10FE0000009810F0FF0008D001280BD002280ED176
:10FE10003046BDE87C40FCF733BB3046BDE87C4053
:10FE2000FDF712B83046BDE87C40FDF759B97CBDFE
:10FE30004801002070B50D4C6068401C606020785F
:10FE40000025411C2170142802D32570FDF7BAFB50
:10FE500000F01AF96088401C80B260800A2804D340
:10FE60006580BDE87040FBF7CBB970BD0000002095
:10FE7000FFF7E0BF10B50121034800F011F8BDE81D
:10FE8000104000F0C9B800000008004000290188B7
:10FE900002D041F0800101E021F080010180704733
:10FEA000C943018270470029018802D041F0010155
:10FEB00001E021F0010101807047002A828901D010
:10FEC0000A4300E08A4382817047000030B502880F
:10FED0001B4C1C4DA0420DD0A8420BD0B0F1804F5E
:10FEE00008D0194B984205D0184B984202D0184BB5
:10FEF000984203D122F070034A881A43154B984266
:10FF000006D0154B984203D022F44073CA881A4396
:10FF100002808A8882850A880285A0420AD0A84287
:10FF200008D00E4A904205D00D4A904202D00D4AA8
:10FF3000904201D1097A01860121818230BD000001
:10FF4000002C014000340140000400400008004043
:10FF5000000C004000100040001400400040014030
:10FF6000004401400048014030B51A4C0021A4F182
:10FF70003405EA8924F81200521C93B2EB81022B5B
:10FF800005D301226A700023EB812A7001E06A78B0
:10FF9000AAB1002234F91230521C92B21944022A3A
:10FFA000F8D301EBD172A1EB6201084400EBD070F1
:10FFB00040100DE034F91250521C294492B29A427A
:10FFC000F8D35B1E91FBF3F2891A084490FBF3F01F
:10FFD00000B230BD5000002001EB81014900012832
:10FFE00011D001EB81000921A0F57A5090FBF1F0CE
:10FFF0000A2190FBF1F201FB120290FBF1F0042ABE
:020000040801F1
:1000000000DD401C704701EBC100052190FBF1F0C1
:1000100000F54860ECE7000070B5FBF7B7FC01287D
:1000200016D1FBF7B9FC0025164C002820DD6188AD
:10003000401E491C618000B2FFF750F8207840B1A3
:1000400001280DD0022803D10020FBF721FF2570E5
:1000500070BD0120FBF71CFF65800120207070BD82
:100060006088B0F5FA7FFAD302202070658070BDF9
:1000700025700020FBF70CFFBDE870400220FFF761
:1000800027B80000180000202DE9F041164F002588
:1000900005EB450617F82600012818D1FBF752FD9D
:1000A00007EB86046168884211D90120607060887E
:1000B00098B1A0F57F41FF3904D0401E0004000C28
:1000C00060800AD0FBF73EFDA168084460606D1CAB
:1000D000EDB20A2DDCD3BDE8F081002007F8260040
:1000E0006060A060F3E700005C0300203EB50C22D6
:1000F0000C4B68460021CC5C4454491C89B29142A7
:10010000F9D30821F8F7FCFF0299814206D10A468B
:10011000054900208A60019A4A603EBDFEF726FE2E
:100120003EBD000000F001085400002010B50C4650
:100130000A46C02100F03CF921460120FEF794FF59
:1001400030210120FEF79EFF044903200870044877
:100150008368191B81600021017310BDCC01002050
:10016000C834002010B586B01549164A002003ABEC
:10017000841894F8E8471C54401CC0B20C28F7D3EC
:1001800000206A460B5C1354401CC0B20C28F9D303
:1001900000980C2248400090019848400190029835
:1001A0004840029003A96846F9F7B4FF002804D13B
:1001B000002211461046FAF777FE06B010BD000087
:1001C000F27F000800F0FF1F7CB50120FEF7A6FBC0
:1001D0000121C805FEF7C6FA01210420FEF7CEFA78
:1001E00014208DF8040002208DF8050000208DF801
:1001F000060001208DF8070001A8FDF7CFFC4FF4A1
:10020000C050ADF8000003248DF8024018200A4DBC
:100210008DF8030069462846FBF7FCF86103ADF84A
:1002200000108DF8024004208DF80300694628462E
:10023000FBF7F0F87CBD00000008014006490548C6
:10024000022208600272064A0448C1E901020068FD
:100250000047000018350020140300205002002041
:10026000AC02002070B50D4D28680D4C2080208810
:100270000C4E31880840400505D50B484068804742
:100280004FF6FF302860208831880840000403D5ED
:10029000BDE87040F8F77EBF70BD0000445C0040D0
:1002A0002C0200202003002050020020FFF7DABFBC
:1002B00010494FF400620A608A140A600D4910392F
:1002C000002808680BD020F4804040F430400860DB
:1002D000086820F4802040F430200860704720F443
:1002E000404040F440500860086820F4402040F44A
:1002F0004030F2E71408014070B500F07F060D466B
:100300003046FBF785FA04463046FBF771FA0146A2
:1003100022462846FDF7E0FE204670BD10B50022BB
:1003200008E0835CA3F16104192C01D8203B8354BD
:10033000521C92B28A42F4D310BDFEE73EB54FF68E
:10034000FF74234640F2371200216846FEF7F8FF9B
:1003500023464FF47A7204216846FEF7F1FF2346E4
:10036000252205216846FEF7EBFF234640F2931253
:1003700002216846FEF7E4FF2346D92201216846A0
:10038000FEF7DEFF234640F2355207216846FEF7AE
:10039000D7FF234640F2052209216846FEF7D0FF29
:1003A000234640F26D4208216846FEF7C9FF3EBD74
:1003B000084B10B5521C520803EB410109D010F84C
:1003C000013B521E10F8014B43EA042321F8043B81
:1003D000F5D110BD006000400EB5154A50780128D7
:1003E00024D00020009001900290BDF80000114B35
:1003F00020F4704110781B7960F34B2121F4907147
:100400009B0963F3871121F01F011031401CADF8E7
:10041000001000F0070010704FF47A70FAF778F8C7
:10042000012050706846F9F788FE0EBD04200EBD0D
:10043000C00100204C3300201CB50C216846FBF79E
:100440002FFB154C0098217AC0B2814203D008B925
:100450000F21A1832072A08B401C80B2A0830F28A3
:1004600004D3012060720020A0830BE00028607A92
:1004700006D0022803D1F9F72BF8032060721CBDC7
:100480000128FCD14FF47A60FEF72EFE0120F9F727
:100490001FF80220F2E70000480100203EB50546A3
:1004A00009216846FBF7BEFB0098C0F3072000282F
:1004B0003AD00020012101FA00F42C4003D1401C65
:1004C000C0B20928F7D3194D287B401C287300209F
:1004D000F9F788F8287BC00711D1012C04D0022C31
:1004E00004D0042C0BD105E011A200E013A20821D6
:1004F000202002E014A208212820FAF799F9287B8D
:1005000006280CD900202873F9F76CF844F0004055
:10051000F7F7C0FF02460B460D20FEF713FEBDE8BD
:100520003E400920F9F766B83EBD000048010020B2
:100530004C6F7720766F6C74210000004869676803
:1005400020766F6C742100004E6F2074697021005A
:10055000FBF7D2BE10B5044645F25550FBF7E0FE5E
:100560000320FBF7D1FE04EB8400C0F38F00FBF700
:10057000D1FEFBF7C1FEFBF7B7FE012010BD000066
:1005800070B542F234110025144C88420AD347F664
:100590001811884203D9A07A401CA07205E0F8F730
:1005A00019FC68B1607A401C6072607A032804D23A
:1005B000A17A032906D3032805D30022084B07E0BC
:1005C0006572A57270BD032905D300224FF08043E8
:1005D0000D20FEF7B7FDFEF7A2FAF1E71C000020A0
:1005E0000000F03F2DE9F041244C00256268A76827
:1005F000D3693E78403316B1012E06D02EE040027A
:10060000E061480220620120387000201C4ED16950
:1006100008E0D4F80CC0375C0CF80170D169491CB3
:10062000401CD1619942F4D3164EE16930880144EF
:10063000E161236A181A2062C00505D1D561A1F5D0
:100640000071E068F9F7C6FF0F4832888168891A9F
:1006500081604FF440510220FEF7CCFC206A18B1B3
:100660000A480078042807D160680121C56100208C
:10067000FEF7CAFEA0680570BDE8F08164000020A6
:1006800068340020CE010020C8340020CC010020B6
:100690000FB4084B10B504A902AA039800F06CFC33
:1006A000044602A9002000F0FEFF204610BC5DF8C1
:1006B00014FB0000A7160108490050EAC12018BF2A
:1006C00004204A0D18BF40F0010040F2FF72B2EB67
:1006D000515F08BF40F00200012808BF05207047A5
:1006E0002DE9F74F144694B00021C4E90211159981
:1006F000079121F00045C9498D4206DC1599C4E9EE
:10070000000117B00020BDE8F08FC549DFF814A341
:10071000A9423CDD0799C44E0029C44FC44A15992B
:10072000534619DDF8F7EEF8554506D0C14AC24BDD
:10073000F8F7E8F8C4E900010AE04FF0D352BE4BE5
:10074000F8F7E0F832463B46F8F7DCF8C4E9000178
:1007500017B00120BDE8F08FF8F733F8554506D003
:10076000B44AB54BF8F72DF8C4E900010AE04FF0A0
:10077000D352B14BF8F725F832463B46F8F721F84B
:10078000C4E9000117B04FF0FF30BDE8F08FAB496E
:10079000A942159978DB21F0004183468846A84A92
:1007A000A84BF7F7E6FD0022A74BF8F70AF8F7F792
:1007B000ABFE0990F7F75DFE06460F469C4A53468E
:1007C000F7F7D7FD43465A46F8F79FF880468A4622
:1007D000984A994B30463946F7F7CBFD2A0D01254B
:1007E0000B9242465346F8F790F8032DC4E90001F6
:1007F00039D00B98C1F30A51401A05EB4511113954
:10080000814230DA9148C346784400EB0510CDF8B8
:100810000CA00C90D0E9002330463946F7F7A9FD2B
:1008200002460B460491069058460399F8F76AF879
:1008300080468A4602460B4658460399F8F762F806
:10084000049B069AF8F75EF883460C9803913946A4
:10085000D0E902233046F7F78CFD5A46039BF8F7A0
:1008600051F86D1CBDE707980028A2BF099817B082
:10087000BDE8F08F616881F000416160099817B0B0
:100880004042BDE8F08FFFE784461598C1F313019D
:10089000C0F30A50A0F2F5304FEA601800F01F06CE
:1008A000C6F12000139000200690079041F4801EAE
:1008B00005206D4676B1664A08EB00017A4452F88D
:1008C000213002EB8101B3404A68139922FA01F109
:1008D000194305E05F4908EB0002794451F8221002
:1008E000A1FB0E27A1FB0C131A449A4234BF01232B
:1008F000002303EB070A05EB8003D3E901B70F449C
:100900008F4234BF0121002193448B4411B19345A0
:1009100002D903E0934501D2012100E00021C3E99F
:1009200001B7514445F82010011EA0F10100C1DCBF
:100930000298059F00F10050800F12900298DDE9A7
:1009400003568000F7F795FD834628460D91F7F78B
:10095000A1FD6FF01D02F8F7FEF8CDE90E0130465B
:10096000F7F798FD6FF03D02F8F7F5F880468A46F4
:100970003846F7F78FFD6FF05D02F8F7ECF80746A1
:10098000424653461191F7F71CFFDDE90E23F7F7B6
:1009900018FF5A460D9BF7F714FF00250E465A46DE
:1009A00028460D9BF7F7AEFFDDE90E23F7F7AAFF08
:1009B00042465346F7F7A6FF3A46119BF7F7A5FFC5
:1009C000DFF898A0244A5346F7F7D3FC0746884639
:1009D000234A244B31462846F7F7CBFC3A46434698
:1009E000F7F7EFFE074688464FF0A84253463146D8
:1009F0002846F7F7BEFC3A464346F7F7E2FE159A5B
:100A000012F0004F04D0129A81F00041524212922B
:100A1000C4E90001129817B0BDE8F08FFB21E93F4F
:100A20007CD90240FB21F93F7370032E8A19A33B46
:100A3000000040543163621A61B4D03DFB2139415A
:100A400083C8C96D305FE43F0000E03FEC2900003F
:100A5000682900004A290000182D4454FB21F93D63
:100A60003326A611460B113C2DE9FF4D21F000481D
:100A700007460C46B8F1795F08DAF7F745FD00281C
:100A800001BF0020324904B0BDE8F08D3A4623464C
:100A900010461946F7F76DFC054602462D480E46EE
:100AA0000B460621784400F05DF82A463346F7F7F6
:100AB00060FCDDE9022382468B4638462146F7F783
:100AC00058FC04460F4652465B4628463146F7F727
:100AD00050FC22463B46F7F715FF07468A464FF083
:100AE000FF3228463146F8F736F81B4A90450ADAB5
:100AF0003A465346F7F706FF04B00022BDE8F04D32
:100B0000134BF7F702BF154A4245A8BFA8F50015D9
:100B10004FF00004B8BF124D22462B46F7F7F2FE05
:100B20000646884622462B4600200949F7F7EAFE8A
:100B300004460D463A46534630464146F7F7E2FE34
:100B400004B022462B46BDE8F04DF7F7DEBE0000AC
:100B50000000F03F202700003333D33F0000E93F7F
:100B60000000D23F2DE9F0414F1E00EBC7010446C3
:100B7000D1E9000115461E4637F006020DD02A467F
:100B80003346F7F7F6FB7F1E04EBC703D3E90023D8
:100B9000F7F717FE37F00602F1D1022F25D0042F08
:100BA00013D0062F18BFBDE8F0812A463346F7F769
:100BB000E0FBD4E90A23F7F704FE2A463346F7F7A9
:100BC000D8FBD4E90823F7F7FCFD2A463346F7F7AC
:100BD000D0FBD4E90623F7F7F4FD2A463346F7F7AE
:100BE000C8FBD4E90423F7F7ECFD2A463346F7F7B0
:100BF000C0FBD4E90223F7F7E4FD2A463346F7F7B2
:100C0000B8FBD4E90023BDE8F041F7F7DABD0000F6
:100C10002DE9FF4D054621F0004084B00C46B0F1AF
:100C2000795F0BDA2846FFF747FD042808BF00F07C
:100C30006FF8284608B02146BDE8F08D2A460B46DD
:100C40001046F7F796FB06460F462A462346F7F767
:100C500090FB804626488A4632463B46052178442A
:100C6000FFF780FF83461098029160B3214A224B20
:100C700040465146F7F77DFBCDE900015A46404614
:100C80005146029BF7F775FB82468846DDE906016F
:100C90004FF0FF32F7F75FFF52464346F7F732FE59
:100CA00032463B46F7F765FBDDE90623F7F72AFEF8
:100CB000DDE90023F7F726FE08B02A462346BDE803
:100CC000F04DF7F722BE0B465A4630463946F7F745
:100CD00050FB084A084BF7F774FD42465346F7F7B6
:100CE00048FB08B02A462346BDE8F04DF7F769BD3A
:100CF0005E260000495555555555C5BF0122F7F7E9
:100D00002ABF0022134610461146F7F701BE000025
:100D1000024A00201107F7F71EBF000001FDFFFF88
:100D200030B502004FF0000303D52D2001230870D9
:100D300052420A2592FBF5F4012004E094FBF5F4FD
:100D400000EB80004000002CF8D10AE092FBF0F4A8
:100D50003034CC5492FBF0F400FB142290FBF5F0FD
:100D60005B1C0028F2D1C854084630BD02E008C818
:100D7000121F08C1002AFAD170477047002001E015
:100D800001C1121F002AFBD1704700000149086011
:100D9000704700002803002010B5044600E0641CE2
:100DA000207800F0DFF80028F9D114F8011B0A467A
:100DB0002D2901D02B2901D114F8011B0020A1F10C
:100DC0003003092B07D800EB800001EB400014F83A
:100DD000011B3038F3E72D2A00D1404210BD00003E
:100DE0002DE9FF5F82B00021DDE90430020DDDF85E
:100DF00040B0034318D044F61050A2F2FF324243F1
:100E00001514119801281FD0A5EB0B00401C5FEAB8
:100E1000000A4FF000064E4FDFF83891B0465046BA
:100E200015D5CAF1000413E0119801244AA3012842
:100E300001D16FEA0B010298119AC0E90031C0E9B3
:100E4000024206B0BDE8F09FCBF10000DFE70446A8
:100E50000021404A491842EB0450CDE9001012E04D
:100E6000E00707D032463B4640464946F7F781FA4D
:100E70008046894632463B4610461946F7F779FACE
:100E800006460F466410002CEAD1DDE90401DDE9D5
:100E90000023BAF1000F06DAF7F76BFA42464B4629
:100EA000F7F767FA05E0F7F733FD42464B46F7F7E9
:100EB0002FFD04460E460022284BF7F701FE03D80B
:100EC0004FF0FF30014607E00022254B2046314617
:100ED000F7F777FCF7F7DCFD102409E0002C0ADBBC
:100EE0000A220023F7F798FB039B30321A55641E41
:100EF00050EA0102F2D1641C039AC4F111031444B4
:100F0000119A012A03D0012208430DD10AE00843B7
:100F100004D000204FF0110B119072E7A3EB0B05EA
:100F20006D1E0DE05B4504DD4FF0000205F101058B
:100F300004E003DA4FF00002A5F10105002AECD02D
:100F400002981199C0E90231C0E9004579E7000033
:100F5000000014400000F03F300000000000F043AB
:100F60000000E03F202805D00D2803D00A2801D03A
:100F700000207047012070472DE9FF4F95B09B4638
:100F80008946064600250FE2252877D1002427460A
:100F9000F84A0121059400E0044316F8013F203B84
:100FA00001FA03F01042F7D130782A2811D06FF0FF
:100FB0002F033078A0F13002092A16D8059A44F0A0
:100FC000020402EB820203EB42021044761C0590FD
:100FD000EFE759F8042B0592002A03DA504244F453
:100FE0000054059044F00204761C30782E2816D167
:100FF00016F8010F44F004042A280DD06FF02F02D8
:101000003078A0F13003092B09D807EB870302EBF6
:101010004303C718761CF3E759F8047B761C307835
:101020006C280FD006DC4C2817D068280DD06A2811
:1010300014D104E0742810D07A280FD10DE044F4C4
:1010400000140AE044F4801401E044F4401472787F
:10105000824202D104F58014761C761C3078662812
:101060000BD013DC582877D009DC002875D0452830
:10107000F6D04628F4D047281AD19DE118E063281D
:1010800035D0642879D0652812D195E1702873D0C5
:1010900008DC6728F1D069286FD06E280DD06F2842
:1010A00006D1B5E073282CD0752875D0782874D077
:1010B0005A46179990476D1C75E1C4F302500228F7
:1010C00009D003280DD0D9F8001004280DD00D60E8
:1010D00009F1040967E1D9F80010EA17C1E90052E3
:1010E000F6E7D9F800100D80F2E70D70F0E719F877
:1010F000041B8DF8001000208DF80100EA46012045
:1011000003E059F804AB4FF0FF3061074FF00001E6
:1011100002D40DE008F101018846B9420FDA80459A
:10112000F8DB1AF808100029F4D108E008F10101F1
:1011300088468142FADB1AF808100029F6D1059892
:101140005B46A0EB080721463846179A00F094FA50
:10115000284400EB080507E04DE029E10DE01AF80E
:10116000010B5A4617999047B8F10108F7D25B4630
:1011700021463846179A13E142E00A220092C4F34E
:1011800002524FF0000A022A08D059F804CB032A71
:101190004FEAEC710AD00DE029E02AE009F10701DD
:1011A00021F00702F2E802C1914609E00FFA8CFC37
:1011B0004FEAEC71042A03D14FFA8CFC4FEAEC7130
:1011C000002907DA0A460021DCF1000C61EB02017C
:1011D0002D2202E0220504D52B228DF804200122C5
:1011E00003E0E20701D02022F7E7904659E00A2108
:1011F00002E010220DE010214FF0000A00910BE0F8
:1012000010224FF0000A44F004040827009203E083
:1012100008224FF0000A0092C4F30252022A05D0BD
:1012200059F804CB0021032A08D009E009F107018D
:1012300021F00702F2E802C1914605E01FFA8CFC9A
:10124000042A01D10CF0FF0C4FF00008220728D52A
:10125000702806D0009B83F0100353EA0A0305D0E0
:101260000EE040228DF80420012208E05CEA010231
:1012700006D030228DF804208DF805000222904619
:10128000009B83F0080353EA0A030AD15CEA0102D7
:1012900001D1620705D530228DF804204FF00108F6
:1012A0007F1E582804D034A003900EA802900DE0B1
:1012B00036A0F9E753466046009AF7F7ADF9844641
:1012C0000398825C0298401E029002705CEA010062
:1012D000F0D1029806A9081A00F1200A600702D589
:1012E00024F4803400E00127574502DDA7EB0A0013
:1012F00000E0002000EB0A01009005984144401AEC
:101300000590E00306D45B462146179A059800F045
:10131000B3F90544002706E001A85A46C05D1799B5
:1013200090476D1C7F1C4745F6DBE0030CD55B4600
:101330002146179A059800F09FF9054404E03020F3
:101340005A46179990476D1C0099481E0090002935
:10135000F5DC08E0029802995A460078491C02918F
:10136000179990476D1CBAF10001AAF1010AF1DC4E
:1013700065E1000009280100303132333435363759
:1013800038396162636465660000000030313233D1
:101390003435363738394142434445460000000071
:1013A00000F058F90544761C307800287FF4ECAD45
:1013B00019B02846BDE8F08F620700D4062709F16E
:1013C000070222F0070CFCE80223E14603F0004884
:1013D0005FEA080C02D00FF2702C0DE05FEA045CAB
:1013E00002D50FF2682C07E05FEAC47C02D00FF24E
:1013F000602C01E0AFF2700C4FF0FF3823F0004397
:10140000CDF850C065280CD006DC452809D0462808
:101410001DD047283DD13DE0662818D067287ED1F1
:1014200038E00021112F01DB112000E0781CCDE90C
:10143000000106A90EA8FFF7D3FCDDE90F010E9A03
:1014400003910021009207F1010A04914DE04FF051
:1014500000400097CDE9011006A90EA8FFF7C0FCD7
:10146000DDE90F0203920E9B11990022DDF80CA01A
:101470000093049211B9791C00EB010AB7EB0A0042
:1014800004D4C0F1FF3007F1010A0490AAEB070071
:10149000019044E0012F00DA01270021112F01DD26
:1014A000112000E03846CDE9000106A90EA8FFF79B
:1014B00097FCDDE90F010E9A03910021049100923F
:1014C000BA4621070CD40399514500DA8A46BAF18D
:1014D000010F05DD009AAAF10101515C302908D005
:1014E000B84202DA10F1040F06DA0121CDE9011049
:1014F00015E0AAF10101E9E7002805DC049901449F
:101500000491AAEB000102E0411C514500DD8A462E
:101510000499401A401C01904FF0004002902007AF
:1015200004D40198504501DBCDF8048000208DF8EB
:101530004F0002980DF14F07B0F1004F25D02B203E
:101540000E9002984FF0020800280CDA40420290F8
:101550002D200E9007E00A210298F7F747F8303166
:10156000029007F8011DB8F10001A8F10108F2DCB2
:1015700002980028EFD1791E0E980870307800F09C
:10158000200040F0450007F8020D12A8C01B00F132
:1015900007081498007800B1012000EB0A010198B7
:1015A00001EBE07105984144401A401E0590E003AC
:1015B00006D45B462146179A059800F05DF805446D
:1015C0001498007818B15A46179990476D1CE0039B
:1015D00024D55B462146179A059800F04DF805443E
:1015E0001CE00498002807DBDDE90301884203DDE5
:1015F0000098405C179901E0179930205A469047AF
:10160000049805F10105401C04900198401E0190CA
:1016100004D12E205A46179990476D1CBAF100014B
:10162000AAF1010ADDDC05E017F8010B5A4617990B
:1016300090476D1CB8F10001A8F10108F4DC5B468D
:101640002146179A0598ABE62D0000002B000000FC
:10165000200000002DE9F041044600251E461746F3
:10166000880404D405E039462020B0476D1C641E70
:10167000F9D52846BDE8F0812DE9F0410446002562
:101680001E469046C80301D5302700E02027880475
:1016900004D505E041463846B0476D1C641EF9D5B7
:1016A0002846BDE8F0810A68531C0B601070704733
:1016B00000B5244B21F0004287B09A42DCBF0022E3
:1016C000134629DD204B9A4208D140B94FF0010062
:1016D000FFF75CFBFFF715FB07B000BD03DBFFF76F
:1016E0000DFB07B000BD02AAFEF7FAFF10F00301E0
:1016F00004BF0DF1080C9CE80F000DD0012001295A
:101700000ED0022914D00DF1080C00909CE80F00B7
:10171000FFF77EFA07B000BDFFF7A6F907B000BDDE
:101720000DF1080C00909CE80F00FFF771FA05E03E
:101730000DF1080C9CE80F00FFF796F907B081F057
:10174000004100BDFB21E93F0000F07F2DE9FF5F74
:101750000D4607463D2100F50070F6F70FFD002805
:101760007ED0401CFFF718FB0404240C01D0012C90
:1017700077D110216846FAF793F900981FFA80F89C
:10178000A04501D04FF001082C8300264FF00A0A33
:101790004FF6FF7B00944FF0000907EB86103D21C8
:1017A000F6F7ECFC00285BD0401CFFF7F5FA84B29A
:1017B000009800B34FF4FA710120FEF70DFC90FB86
:1017C000FAF0A04208DC4FF47A610120FEF704FC35
:1017D00090FBFAF0A04201DA4FF00109904800783E
:1017E00030B3B9F1000F23D0052E21D2DFE806F087
:1017F000091741434500A4F13200B0F5AF7FEBD8A3
:10180000ECE702210CE004EB8400B1EB400F0FD1B8
:10181000287EFEF7E1FB90FBFAF084B208E003219A
:1018200002A8FAF73DF90298B8F1000F81B2EAD1A7
:10183000009820B34FF4FA710120FEF7CDFB90FB26
:10184000FAF0A0420DDC4FF47A610120FEF7C4FBF0
:1018500090FBFAF0A04204DBBEB1012E1BD001E0E8
:10186000BAE08FE0022E1CD0032E20D0042E24D00C
:1018700028E00421D4E70521D2E71621D0E7A4F11E
:101880003200B0F5AF7F7DD8E6E704EB84010BEAC8
:101890004100A88016E004EB84010BEA4100E880D7
:1018A00010E004EB84010BEA410028810AE004EB1C
:1018B00084010BEA4100688104E004EB84010BEA37
:1018C0004100E883761CB6B2052EFFF464AF3D21DB
:1018D00007F5A070F6F752FC00287DD0401CFFF7FA
:1018E0005BFA80B2A0F13C014FF46B74A14249D283
:1018F00068823D2107F5C070F6F740FC00286BD0E8
:10190000401CFFF749FA80B2A0F13C01A14239D254
:10191000A8823D2107F5E070F6F730FC002879D069
:10192000401CFFF739FA80B2411E0A2971D2288281
:101930003D2107F51070F6F721FC00286AD0401C05
:10194000FFF72AFA80B2411E022962D2E8823D21C5
:1019500007F52070F6F712FC00285BD0401CFFF75B
:101960001BFA80B2411E192953D228843D2107F564
:101970003070F6F703FC00284CD0401CFFF70CFA3F
:10198000000400E045E0000C02D0C11E042940D252
:1019900068833D2107F54070F6F7F0FB002839D049
:1019A000401CFFF7F9F980B2A0F6B831B1F57A7FA3
:1019B0002FD8A8833D2107F55070F6F7DFFB0028EC
:1019C00028D0401CFFF7E8F980B2012821D86884AC
:1019D0003D2107F5607000E01CE0F6F7CFFB002822
:1019E00018D0401CFFF7D8F980B22D2811D8411E1D
:1019F00011290ED3A8843D2107F57070F6F7BEFBC0
:101A0000002807D0401CFFF7C7F980B2411E052906
:101A100003D3002004B0BDE8F09FE8840120F9E77B
:101A200064000020FCF7C2FE4FF40040FCF7AAF867
:101A30004FF0E0204BF67F3141612C4AF02182F8D3
:101A4000141D0021816107210161FAF705FBF9F7F7
:101A5000D3FBF8F73BFD0020FEF72AFC4FF496700D
:101A6000F8F742FD0120FEF723FCFEF7ADFBFEF781
:101A7000E5FBF8F75FFDFCF753FEF7F761FFFCF7B6
:101A800053FFFDF765FEF8F7F1FEFBF785FDFEF766
:101A900069FBFCF71DFEFAF703FAF7F7ABF82F2105
:101AA0006320FAF7A5FC4FF4FA70F8F71DFDFCF778
:101AB0009FFDFEF743FC4FF47A70FEF74BFDF7F7FE
:101AC000A1FC80B2F6F7E6FC02460B460020FDF7CB
:101AD00039FBFEF73DFDF9F753FF012803D1F9F774
:101AE00055FFFAF7FBF9FEF767F9F2E70FE000E0C0
:101AF0000FB42DE9FC474FF0000705003C4606D027
:101B00000CAEEA464FF00A084FF02E0916E000200E
:101B1000BDE8FC075DF814FB25280CD17F1CC85DCF
:101B2000632806D064281AD0662826D0732802D1EC
:101B30000BE016F8040B2855641C7F1C0B99C85D3C
:101B40000028E9D128552846E2E704CE002002E02B
:101B50002955401C641C115C0029F9D1EDE701CE28
:101B60006946FFF7DDF80020524602E02955401C87
:101B7000641C115C0029F9D1DFE701CE411E082960
:101B8000DBD909395929D8D95A39B1F5617F1AD227
:101B9000414690FBF1F208FB120290FBF1F030326B
:101BA000EA7090FBF1F208FB120290FBF1F0303288
:101BB000AA7090FBF8F208FB1200303085F8019013
:101BC00028700424B9E7A0F57A7142F227329142D5
:101BD000B3D8414690FBF1F208FB120290FBF1F002
:101BE00030322A7190FBF1F208FB120290FBF1F007
:101BF0003032EA7090FBF1F208FB120290FBF1F038
:101C000085F8029030326A7090FBF1F208FB120006
:101C100030302870052490E7034600F001000121D0
:101C2000420023FA01F000F001001043491C202972
:101C3000F6D370472DE9F04106460F46F6F7D7FE7A
:101C4000041E0D4618BF0120284320F00040C0F1BB
:101C50007F6000F1E040C00F0ED0301C18BF0120A3
:101C6000384320F00040C0F17F6000F1E040C00F39
:101C700004BF0120FFF78AF820462946BDE8F0811D
:101C8000007F3E1C08002C36FBFB362C00E038247D
:101C9000322A2A322438E000000704040404040431
:101CA00004040700AED552A80FC8D30040A18D147C
:101CB000DA0281E0D9F1DB30A4A6AFAED552A80F8D
:101CC000C8D30040A18D14DA0281E0D9F1DB30A441
:101CD000A6AFAED552A88F0833E080218D14DA026A
:101CE000816019111BB0A4A62F6E955228CF28131E
:101CF0008040A18D145AC281E0D9F1DB30A4A6AF97
:101D0000AED552A80FC8D30040A18D14DA0281E0ED
:101D1000D9F1DB30A4A6AFAED552A80FC8D300408E
:101D2000A18D14DA0281E0D9F1DB30A4A6AFAED5E3
:101D300052A80FC8D30040A18D14DA0281E0D9F176
:101D4000DB30A4A6AFAED552A80FC8D30040A18DFA
:101D500014DA7ABDFED6F6DC2F9BD950D1EB4CA617
:101D600008CFD403596D6B66E21E8FE7DEFEC40F09
:101D7000DB59D190CA5DAF0FC8D30040A18D14DAF2
:101D80000281E0D9F1DB30A4A6AFAED552A80FC8CE
:101D9000D30040A18D14DA0281E0D9F1DB30A4A692
:101DA000AFAED552A80FC8D30040A18D14DA02817E
:101DB000E0D9F1DB30A4A6AFAED5A2C8CF4853C05E
:101DC00020518D14DA02911029E1DB30A4A6BF5E08
:101DD00095D2281F38C30040A19DE42A1281E0D982
:101DE000C12BD024465F4E55B2583FC8D30040A106
:101DF0000DD4AA724160D9F1DB30A4965F5E45C272
:101E000058EFC8D30040A18DE42AB2315069F1DB0C
:101E100030A4A6AFAED552A80FC8D30040A18D14F0
:101E2000DA0281E0D9F1DB30A4A6AFAED552A80F1B
:101E3000C8D30040A18D14DA028DEFD9F0D833A5B4
:101E4000A6A0A2D552A807C7DC0840A18D14D60DC4
:101E500081E0D8F2D43CA4A6AFA6DA5DA00FC8D327
:101E60000041AE8217DA018EEFD8F1DB30A4AAA1CF
:101E7000A9D650AA0CCFDD0C40A18D1AD50381E163
:101E8000DEFFD738A4A6AFA1DA5EA403C4DF0C48F6
:101E9000A18D14DA0281E0D9F1DB30A4A6AFAED572
:101EA00052A80FC880AE80D5805280A8800F80C80D
:101EB00080D38000804080A1808D801480DA8002F1
:101EC000808180E080D980F180DB803080A480A692
:101ED00080AF00FCF8F0E0C08000001F0F07030196
:101EE0000000AE001040B08140A0A6A81FC8D300DB
:101EF000D580D922DA12DB408D14AF00560E4B0E7E
:101F0000410E360E2B0E1F0E140E080EFD0DF00D99
:101F1000E40DD80DCB0DBE0DB10DA40D960D890DA0
:101F20007B0D6D0D5E0D500D410D320D230D140D09
:101F3000040DF50CE50CD50CC40CB40CA30C920CE0
:101F4000810C700C5F0C4D0C3B0C290C170C040C15
:101F5000F20BDF0BCD0BB90BA60B930B800B6C0BAD
:101F6000580B440B300B1C0B080BF30ADF0ACA0A90
:101F7000B60AA10A8C0A770A620A4C0A370A220AB0
:101F80000C0AF709E109CC09B609A0098B09750902
:101F90005F09490933091D090809F208DC08C60868
:101FA000B0089A0885086F08590843082E081808D1
:101FB0000308ED07D807C207AD07980783076E0728
:101FC000580744072F071A070507F106DD06C8065C
:101FD000B406A0068C067806650651063E062B065A
:101FE00017060406F205DF05CC05BA05A805960517
:101FF0008305720560054F053D052C051B050A0587
:10200000F904E904D804C804B804A80498048904AD
:1020100079046A045B044C043D042F042004120478
:102020000404F603E803DB03CD03C003B303A603F4
:1020300099038C038003740367035B034F0344031A
:1020400038030000F8FFFFFFFFFFFFFFEB3C904D60
:1020500053444F53352E3000020108000200025055
:1020600000F80C000100010000000000000000006A
:10207000000029A298E46C4E4F204E414D4520208F
:102080002020464154313220202033C98ED1BCF06B
:102090007B8ED9B800208EC0FCBD007C384E247DDC
:1020A000248BC199E83C01721C83EB3A66A11C7C2D
:1020B00026663B07268A57FC750680CA02885602A8
:1020C00080C31073EB33C98A461098F7661603462F
:1020D0001C13561E03460E13D18B7611608946FCE5
:1020E0008956FEB82000F7E68B5E0B03C348F7F372
:1020F0000146FC114EFE61BF0000E8E60072392681
:10210000382D741760B10BBEA17DF3A66174324EF9
:10211000740983C7203BFB72E6EBDCA0FB7DB47D3A
:102120008BF0AC9840740C487413B40EBB0700CD10
:1021300010EBEFA0FD7DEBE6A0FC7DEBE1CD16CD35
:1021400019268B551A52B001BB0000E83B0072E81B
:102150005B8A5624BE0B7C8BFCC746F03D7DC74690
:10216000F4297D8CD9894EF2894EF6C606967DCB30
:10217000EA030000200FB6C8668B46F86603461CCB
:10218000668BD066C1EA10EB5E0FB6C84A4A8A4633
:102190000D32E4F7E20346FC1356FEEB4A525006BA
:1021A000536A016A10918B4618969233D2F7F691D2
:1021B000F7F64287CAF7761A8AF28AE8C0CC020A92
:1021C000CCB80102807E020E7504B4428BF48A56AC
:1021D00024CD136161720B40750142035E0B49759A
:1021E00006F8C341BB000060666A00EBB04E544C79
:1021F00044522020202020200D0A52656D6F766504
:10220000206469736B73206F72206F74686572202D
:102210006D656469612EFF0D0A4469736B206572F8
:10222000726F72FF0D0A507265737320616E7920B0
:102230006B657920746F20726573746172740D0A16
:1022400000000000000000ACCBD855AA4553313542
:102250005F415050202020080000000000000000D6
:1022600000007B865B5300000000000000000000BF
:102270000080C06030180C0000000000000000006A
:10228000000103060C1830000000000000000000F0
:10229000000C183060C0800000000000000000004A
:1022A0000030180C0603010000000000060909E6D2
:1022B000F80C040202020202041E000000000007E3
:1022C0001F302040404040402010000000001824F3
:1022D000241802FE828282E2061E00000000000036
:1022E0000000203F2000000300000000000000006C
:1022F00000000000002F000000000700070000148D
:102300007F147F1400242A7F2A120062640813239A
:1023100000364955225000000503000000001C2231
:102320004100000041221C000014083E081400086F
:10233000083E0808000000A060000008080808081F
:10234000000060600000002010080402003E5149B7
:10235000453E0000427F4000004261514946002155
:1023600041454B31001814127F100027454545396F
:10237000003C4A49493000017109050300364949CA
:10238000493600064949291E000036360000000083
:1023900056360000000814224100001414141414CE
:1023A0000000412214080002015109060032495977
:1023B000513E007C1211127C007F49494936003E93
:1023C00041414122007F4141221C007F494949414E
:1023D000007F09090901003E4149497A007F080848
:1023E000087F0000417F4100002040413F01007F05
:1023F00008142241007F40404040007F020C027FD1
:10240000007F0408107F003E4141413E007F0909E2
:102410000906003E4151215E007F09192946004608
:10242000494949310001017F0101003F4040403FDF
:10243000001F2040201F003F4038403F0063140829
:102440001463000708700807006151494543000004
:102450007F41410000552A552A55000041417F0027
:10246000000402010204004040404040000001021C
:102470000400002054545478007F48444438003805
:102480004444442000384444487F0038545454188D
:1024900000087E0901020018A4A4A47C007F08049F
:1024A00004780000447D4000004080847D00007F6F
:1024B000102844000000417F4000007C041804788C
:1024C000007C0804047800384444443800FC242488
:1024D00024180018242418FC007C08040408004870
:1024E0005454542000043F444020003C4040207C91
:1024F000001C2040201C003C4030403C0044281080
:102500002844001CA0A0A07C004464544C44141433
:102510001414141418D8E0301818181800070F18DD
:1025200030303030181800F8F81818180000003F44
:102530003F03030300000000000000000000000053
:1025400000000000000000F8000000000000003360
:102550003000000000100C06100C06000000000007
:102560000000000040C07840C0784000043F0404F0
:102570003F040400007088FC08300000001820FFB1
:10258000211E0000F008F000E018000000211C03EC
:102590001E211E0000F00888700000001E21232468
:1025A0001927211010160E00000000000000000086
:1025B00000000000000000E0180402000000000716
:1025C0001820400000020418E0000000004020181D
:1025D00007000000404080F0804040000202010FF0
:1025E00001020200000000F0000000000101011FD4
:1025F00001010100000000000000000080B0700038
:1026000000000000000000000000000000010101C7
:102610000101010100000000000000000030300056
:102620000000000000000000806018040060180630
:102630000100000000E010080810E000000F10206A
:1026400020100F00001010F8000000000020203FB4
:10265000202000000070080808887000003028243E
:1026600022213000003008888848300000182020DF
:1026700020110E000000C02010F800000007042404
:10268000243F240000F80888880808000019212049
:1026900020110E0000E0108888180000000F1120A3
:1026A00020110E0000380808C83808000000003F5C
:1026B000000000000070880808887000001C2221BB
:1026C00021221C0000E010080810E0000000312268
:1026D00022110F00000000C0C00000000000003008
:1026E000300000000000008000000000000080605A
:1026F00000000000000080402010080000010204DB
:1027000008102000404040404040400004040404C1
:10271000040404000008102040800000002010087D
:1027200004020100007048080808F00000000030B2
:1027300036010000C030C828E810E0000718272440
:1027400023140B000000C038E0000000203C2302EE
:102750000227382008F8888888700000203F202051
:1027600020110E00C0300808080838000718202083
:102770002010080008F808080810E000203F20207A
:1027800020100F0008F88888E8081000203F20205B
:102790002320180008F88888E8081000203F20004F
:1027A00003000000C0300808083800000718202087
:1027B000221E020008F808000008F808203F210146
:1027C00001213F20000808F8080800000020203FF1
:1027D0002020000000000808F8080800C080808061
:1027E0007F00000008F888C028180800203F20015A
:1027F0002638200008F8080000000000203F2020B4
:102800002020300008F8F800F8F80800203F003FCA
:10281000003F200008F830C00008F808203F2000E2
:1028200007183F00E01008080810E0000F102020F3
:1028300020100F0008F808080808F000203F2101C8
:1028400001010000E01008080810E0000F1824241F
:1028500038504F0008F8888888887000203F200092
:10286000030C302000708808080838000038202148
:1028700021221C00180808F8080818000000203F52
:102880002000000008F808000008F808001F2020B9
:1028900020201F000878880000C83808000007388A
:1028A0000E010000F80800F80008F800033C0700DB
:1028B000073C0300081868808068180820302C0343
:1028C000032C30200838C800C83808000000203F1A
:1028D0002000000010080808C83808002038262109
:1028E00020201800000000FE020202000000007F0D
:1028F00040404000000C30C000000000000000011B
:102900000638C00000020202FE0000000040404005
:102910007F0000000000040202020400000000002A
:1029200000000000000000000000000080808080A7
:10293000808080800002020400000000000000008F
:102940000000000000008080808000000019242228
:1029500022223F2008F8008080000000003F112064
:1029600020110E000000008080800000000E112069
:1029700020201100000000808088F800000E112047
:1029800020103F200000808080800000001F222255
:1029900022221300008080F0888888180020203FC1
:1029A000202000000000808080808000006B9494D4
:1029B0009493600008F8008080800000203F210090
:1029C00000203F2000809898000000000020203F59
:1029D00020200000000000809898000000C0808047
:1029E000807F000008F8000080808000203F2402E3
:1029F0002D302000000808F8000000000020203FD3
:102A0000202000008080808080808000203F200087
:102A10003F20003F8080008080800000203F210018
:102A200000203F200000808080800000001F2020C8
:102A300020201F00808000808000000080FFA120F7
:102A400020110E000000008080808000000E112008
:102A500020A0FF80808080008080800020203F2197
:102A6000200001000000808080808000003324244A
:102A700024241900008080E0808000000000001FF6
:102A8000202000008080000000808000001F2020A7
:102A900020103F20808080000080808000010E3068
:102AA0000806010080800080008080800F300C03C9
:102AB0000C300F0000808000808080000020312ECC
:102AC0000E312000808080000080808080818E70A8
:102AD0001806010000808080808080000021302C5A
:102AE0002221300000000000807C02020000000073
:102AF000003F404000000000FF0000000000000018
:102B0000FF0000000002027C800000000040403F07
:102B100000000000000601010202040400000000A1
:102B200000000000000000C0F0F8F81C0C040404D1
:102B30000C3CF8F8F0800000000000FFFFFFFF00F1
:102B4000000000000000FFFFFFFF00000000000089
:102B50000307070E0C0808080C0F07070300000006
:102B60000000000008080808F8FCFCFC0000000059
:102B7000000000000000000000000000FFFFFFFF59
:102B8000000000000000000000000000000808082D
:102B90000F0F0F0F0808080800000000000060F089
:102BA000F8D8CC84040404040C0CFCF8F8F04000C1
:102BB000000000000181C1E06030381C0C0F0707E5
:102BC000030100000000000C0F0F0D0C0C0C0C0C8E
:102BD0000C0C0C0C0F0F000000000070F8F8EC4417
:102BE000040404040C1CFCF8F8F00000000080C091
:102BF000C0C0C000040404040E0BBBFBF9F0C0000D
:102C00000000010307070C0808080808080C0F0754
:102C100007030000000000000000000080C0E0F892
:102C2000FCFCFCFC000000000000C0F0B89C8E879B
:102C3000838180FFFFFFFFFF808080000000000095
:102C4000000000000808080F0F0F0F0F0808080009
:102C5000000000E0FCFC0C0C0C0C0C0C0C0C0C0C24
:102C60000C0000000000008F8F8F8602020301031A
:102C70000306FEFEFCF8200000000007070F0D0809
:102C8000080808080C0E070703010000000000C038
:102C9000F0F8F81C0C040404047C78783000000080
:102CA000000000FFFFFFFF04060202020206FEFC16
:102CB000FCF86000000000010307070E0C0808087C
:102CC000080C0F07070100000000007C7C1C0C0CA6
:102CD0000C0C0C0C0C8CCCEC3C1C0C000000000010
:102CE0000000000000E0F8FEFF0701000000000007
:102CF0000000000000000000000F0F0F0F00000098
:102D000000000000000000F0F8F8FC0C04040404CB
:102D10000C1CFCF8F0E000000000C0F0F1FB3B0FE1
:102D20000F060E0E1E3B7BF1F1E0C0000000010318
:102D300007070E0C08080808080C0E070703010017
:102D4000000000E0F0F8FC1C0C0404040C1CF8F873
:102D5000F0C00000000000070F9F9F181010101017
:102D60001018FFFFFFFF1C000000000007070F0BFB
:102D7000090808080C0E0707030000000000000007
:102D80000000000000000000000000000000000043
:102D90000000000000000000000000000000000033
:102DA0000000000000000000000000000000000023
:102DB0000000000000000000000018242498C060FB
:102DC00030180C0C0C0C0C18306040000000000097
:102DD0001E7FF380000000000000000000808000E3
:102DE000000000000000000103060C0C0C0C0C0697
:102DF0000301000000182424180000FCFCFC1C1C2B
:102E00001C1C1C1C1C1C000000000000000000FF1B
:102E1000FFFF1C1C1C1C1C1C1C00000000000000F0
:102E20000000003F3F3F00000000000000000000E5
:102E30000000000000000000000000000000000092
:102E400000000000000000181818181818181818AA
:102E500018181818180000000000000000000000FA
:102E6000000000000000000000000000A00078004A
:102E7000500032001E0000806010080464940404B6
:102E8000B44C04848484848484040404040404040A
:102E900084442464A42424242424242424E404082E
:102EA000106080000000000718204080828180822E
:102EB000828585888F8888888F85858585858585A5
:102EC0008D95A7B0AFA0A0A0A0A0A0A0A0BF80405B
:102ED0002018070000000000806010080484C4E48B
:102EE000E4E4E4C4840404040404040404040404C2
:102EF000040404040404040484C4E4E4E4E4C48492
:102F000008106080000000000718204080848C9C1E
:102F10009C9C9F8F87838383838383838383838323
:102F20008383838383838383878F9F9C9C9C8C84F0
:102F3000402018070000000000F8F8808080F800AA
:102F40008040404040800080404040408000004041
:102F500040F840400000D000408040404080008069
:102F60004040408000000000001F1F0101011F00C1
:102F70000F121212120B000C121212120F1000007C
:102F8000000F100800001F00001F0000001F004776
:102F90008888887F000000E0F0101020000080800A
:102FA000808000008080F08080008080F080800041
:102FB000A0008000808080800000008080808000F1
:102FC000000000000000000811111F0E000F121277
:102FD00012120B0000000F10080000000F10080074
:102FE0001F00001F000000001F004F909090907F76
:102FF00000000000000000008060100804040404C9
:1030000084C464C4840404040404040404040404A0
:103010000404040404040404040404040404040470
:10302000081060800000000007182040A0B0B8BE63
:10303000BFBFA8BFBFBEB8B0A080808080808080A6
:103040008080808080808080808080808080808080
:103050004020180700004060504844444444444421
:103060004444444444444444444444444444444420
:103070004444444444444444444444444444444410
:103080004444444444444444444444444444444400
:10309000444444444444444424140C0400001018A0
:1030A0008CC663C68C1810000000426331180C18DF
:1030B00031634200FFFFFF0FFFFFFF0F120100020D
:1030C000EF020140160401DC0002010203010902C3
:1030D0006200030100C03209040000020806500427
:1030E0000705810240000007050202400000080BAE
:1030F00001020202010109040100010202010005AE
:103100002400100105240100010424020205240604
:103110000001070584030800FF09040200020A00F9
:10312000000007050502400000070583024000007B
:1031300004030904280365002D00440065007300A2
:1031400069006E00670049006E00740065006C0045
:103150006C006900670065006E007400260354006F
:10316000530031003000310020004D006100730039
:1031700073002000530074006F007200610067004C
:1031800065001C0365002D004400650073006900A4
:1031900067006E0020004D00610073007300008026
:1031A0000202200000004D696E692044534F4469BB
:1031B000736B202020202020202020202020202071
:1031C00020200000000000004C5555555555A53FE6
:1031D0007751C1166CC156BF9015CB19A001FA3EAC
:1031E000AD529C804F7E92BEC4B1B4BD9EEE213ED6
:1031F000D43888BEE9FAA8BD00004054FB21F93F4D
:103200003163621A61B4D03D0000601A61B4D03DF0
:103210007370032E8A19A33B0000002E8A19A33B6A
:10322000C14920259A837B3900000000000000007E
:103230006E83F9A22915444ED15727FCC0DD34F521
:10324000999562DB4190433CAB6351FE61C5BBDEA7
:103250003A6E24B7E0D24D42EA2E49061C92D109BB
:103260001CEB1DFE3EA729B1F53582E88444BB2E38
:1032700026709CE9417E5FB439D69139F439538385
:103280008B5F849C3B28F9BDFF97F81F0F9805DEE4
:103290008B112FEF1F6D0A5ACF7E366DB709CB27E2
:1032A000663F464F2DEA5F9EC7BA27757BF1E5EB77
:1032B000F739073DEA92528AB15FFB6B085D8D1FBB
:1032C000A6F810111111813FD561C119A0012ABFC3
:1032D0007DFEB157E31DC73EEB9C2B8AE6E55ABE47
:1032E0007CD5CF5A3AD9E53D202023286D563A3374
:1032F0003330307E34303030290D0A002020202336
:1033000028317E3130290D0A0000000020202023C2
:1033100028433A35307E34303020463A3132327EDE
:10332000373532290D0A0000202328433A35307EF4
:1033300034303020463A3132327E373532290D0A68
:10334000000000002020202328317E3235290D0A7C
:1033500000000000202020202328317E35290D0A7E
:103360000000000020202023285365633A36307E79
:10337000393939290D0A0000202023285365633A82
:1033800036307E393939290D0A00000020202020EE
:103390002328303A4320313A46290D0A0000000024
:1033A00020202328303A4F464620313A204F4E29DC
:1033B0000D0A0000202020202328303A44432033E7
:1033C0007E363A337E3653290D0A00002020202015
:1033D000202328303A4F46462031387E34353A3162
:1033E000387E343557290D0A00000000202023289C
:1033F000313A526967687420323A4C656674290D17
:103400000A00000054315F54656D703D3330300068
:103410004D696E566F6C743D3335303000000000DE
:1034200054656D70537465703D31300054325F5493
:10343000656D703D3333300049646C6554696D656A
:103440003D32343000000000536C7054656D703DA7
:103450003235300054335F54656D703D3335300084
:10346000536C7054696D653D31383000426F6F7335
:103470007454656D703D333830000000506F7765CF
:10348000725372633D30000054656D70556E6974FF
:103490003D3000004C6F7743757272656E743D303D
:1034A00000000000504450774D61783D300000002E
:1034B000446973706C61794469723D3100000000A9
:1034C0004261636B6C696768743D33004D73656E70
:1034D000556E69743D330000506F776572537263A7
:1034E0000000000049646C6554696D6500000000CF
:1034F000536C7054696D650054656D7053746570DC
:103500000000000054315F54656D700054325F5408
:10351000656D700054335F54656D7000536C70546A
:10352000656D7000426F6F737454656D70000000BC
:10353000446973706C617944697200004261636B25
:103540006C696768740000004D73656E556E697430
:103550000000000054656D70556E69740000000035
:103560004D696E566F6C74004C6F7743757272655F
:103570006E740000504450774D6178009C3501080E
:10358000000000202C030000848B00080437010891
:103590002C0300200C4200007C0D010801105AFF92
:1035A00001810233027755AA5AA59001440188137C
:1035B0001390301B20B00413902E0214201E0435EB
:1035C00001080C041A14041A1C041A24041EF034F2
:1035D0000108E4041A3C0C1A54041A30041AF810B6
:1035E0001AD8041A600C1A68041A74041A48041AC7
:1035F00004141A2C041A54041A48042A6C241904BA
:103600001A38041AC0041A88041AB0041A20041ABA
:103610007C041A10041A94041AA4041ACC04CB0CC7
:1036200033041A28041A64041A78041EFC320108B0
:103630008C081AEC041A44041AB4041AE8141AA0E8
:10364000081ACC041A540429EF46010104020302AB
:1036500016FF4009B80BE40CAC0DC40912032AB4E0
:103660003251061AAC0DD80E0A395B592B69070185
:1036700021141A034D12691A6E0412771261127224
:10368000B26513E1A9140883DB5B08E908E9049A31
:10369000E5189AED0CD12AC28A120836BC3001080E
:1036A000121ACE083262137DD9140811D81B08658E
:1036B000081A79041301D71B08B5041AA9041A7D46
:1036C000041A71041A890441324036303101080469
:1036D0001A340832281A5C08322613D80133201A0B
:1036E0001A8210321C1A066F2984CB89DAAC1AB5FB
:1036F00064690C1ABD1C419203E2066270D20A3959
:04370000330224026A
:04000005080080ED82
:00000001FF
